:105A4D00755606123E7C202B04E54470F9123EC5B6
:105A5D00755606123E3C80E822755604123E7CE5D2
:105A6D004470FC123EC5755604123E3C7F0112383F
:105A7D00E17E007FFF8F051257CBDFF97E007FFFA0
:105A8D00900000C007125808EFF0A3D007DFF422F2
:105A9D00755601123E7CE54470C5123EC575560122
:105AAD00123E3C227557011238E178083029FDE588
:0B5ABD004924301238B2C229D8EA2276
:102E8C007584008537D28538D37584018539D28510
:102E9C003AD3E4F538F537300006853B37853C38B6
:102EAC0030010CE537253DF537E538353EF5383042
:102EBC000210E548852EF0A42537F537E5F03538B6
:102ECC00F538300310E50A8531F0A42537F537E5E0
:102EDC00F03538F538300410E5118530F0A425377D
:102EEC00F537E5F03538F538E4F53AF539300810B2
:102EFC00853B39853C3AE53CC39535400385353AED
:102F0C00300916E53EC39534400385353EE5392539
:102F1C003DF539E53A353EF53A300A10E548852E4F
:102F2C00F0A42539F539E5F0353AF53A300B10E5D2
:102F3C000A8531F0A42539F539E5F0353AF53A3002
:102F4C000C10E5118530F0A42539F539E5F0353A4A
:102F5C00F53A300D10E518852FF0A42539F539E533
:102F6C00F0353AF53A300E10E52C8533F0A42539BE
:102F7C00F539E5F0353AF53A300F10E52D8532F09C
:102F8C00A42539F539E5F0353AF53AE53AC39536E5
:102F9C00400385363A2290308E302D03122FC430E8
:072FAC002E03122FD4303078
:102FB3000312303B302F03122FF730310312304B03
:102FC30022E50B2509F50BE50C3508F50C93F50AFD
:102FD30022E512250EF512E513350DF51393C313F0
:102FE300F8E5142510F514E515350FF51593C313FE
:102FF30028F51122103908203A3C303D238026D28F
:103003003A203B0E303C2FC23AC23DC23B756C00A6
:103013008024203C21C23AD23DD23B756C008016FD
:1030230090318E80039031D6E56C93F52C056CE5D9
:103033006CB44802D23A2222E5192517F519E51A8C
:103043003516F51A93F51822103E08203F3C3042FE
:10305300238026D23F20400E30412FC23FC242C2BE
:1030630040756D008024204121C23FD242D2407579
:103073006D00801690323E800390321EE56D93F50D
:103083002D056DE56DB44802D23F227F8285888C81
:103093008F9295989B9EA1A4A7AAADB0B3B6B9BBD6
:1030A300BEC1C3C6C9CBCED0D3D5D7D9DCDEE0E20F
:1030B300E4E6E7E9EBEDEEF0F1F2F4F5F6F7F8F913
:1030C300FAFBFCFCFDFDFEFEFEFEFEFEFEFEFEFE2A
:1030D300FDFDFCFCFBFAFAF9F8F7F6F4F3F2F0EF76
:1030E300EDECEAE8E7E5E3E1DFDDDBD8D6D4D1CFE9
:1030F300CDCAC8C5C2C0BDBAB7B4B2AFACA9A6A346
:10310300A09D9A9794908D8A8784817E7A77747133
:103113006E6B6865625F5C595653504D4A47444233
:103123003F3C393734322F2D2A282624211F1D1BDB
:103133001918161412110F0E0C0B0A0807060504B2
:10314300040302020101000000000000000000006F
:1031530001010202030405060708090A0B0D0E10FC
:1031630011131516181A1C1E20222427292B2E3062
:103173003335383A3D404245484B4E515456595CDD
:10318300606366696C6F7275787B7FFEFEFEFEFD81
:10319300FCFCFBFAF8F7F6F4F3F1EFEDEBE9E7E407
:1031A300E2DFDCDAD7D4D0CDCAC6C3BFBCB8B4B073
:1031B300ACA8A39F9B96928D89847F7A75706B666A
:1031C300615C57514C47413C37312C26211B16106B
:1031D3000B050000050B10161C21272C32373D422E
:1031E300484D53585D62686D72777C81858A8F94F0
:1031F300989DA1A5AAAEB2B6BABEC1C5C8CCCFD25E
:10320300D5D8DBDEE1E3E6E8EBEDEFF1F2F4F6F738
:10321300F8F9FBFBFCFDFEFEFEFEFE000C19263357
:103223003F4C5864707B86919CA6AFB8C1C9D1D876
:10323300DEE4EAEFF3F6F9FCFDFEFEFEFDFCFAF731
:10324300F4F0EBE6E0DAD4CCC5BCB4ABA1978D8344
:0B325300786D61554A3D3125180C00D4
:10380F00D2F4C2F5C2F675840F85F0C812363F7434
:10381F000312385E123633740312385E12361612E4
:10382F003616740312385E123616740212385E1290
:10383F00361674281238CA74061238CA740E123823
:10384F00CA74011238CA12363374801238CA22C0B1
:10385F0000A2E092F3A2E192F2A2E292F1A2E3922D
:10386F00F0D2F475840F85F0C8C2F47830D8FE8595
:10387F00F0C87830D8FED00022C00075840FA2E4C3
:10388F0092F3A2E592F2A2E692F1A2E792F0D2F4BD
:10389F0085F0C8C2F47830D8FE85F0C87830D8FEED
:1038AF00D00022EF75840FD2F5C2F685F0C812381A
:1038BF008812361612385E1236162275840FC2F52C
:1038CF00C2F685F0C812388812361612385E1236D4
:1038DF001622EF14A2E492E6C2E4D2E71238CA220B
:1038EF00740F1238CA22740D1238CA227F0112388F
:1038FF00E178107F201238B2D8F9227F111238E107
:10390F0078107F201238B2D8F9227F011238E1786F
:10391F00207F201238B2D8F922C0077F018004C05F
:10392F00077F111238E1D007C082C083C007EF753F
:10393F00F0109039591236577810E493FF1238B2BD
:09394F00A3D8F7D007D083D08281
:10395800222020202020202020202020202020205D
:1039680020303132333435363738394142434445D3
:1039780046202020525334323220544553542020BC
:1039880020202020525332333220544553542020D3
:103998002020205445535420204641494C4544207A
:1039A800202020544553542020504153534544204F
:1039B800202020454550524F4D2054455354202037
:1039C80020204155582052454C41592054455354C4
:1039D8002020205055534820544F2054414C4B2010
:1039E8002054455354203320434841522F535542C5
:1039F800205445535420464958454420535452496D
:103A08004E5445535420564152494220535452492A
:103A18004E464143544F52592044454641554C5413
:103A28002050524F4752414D4D494E47204D4F442B
:103A38004553494D504C45582052455045415445F1
:103A4800522020205245434F5244494E47202020BF
:013A5800204D
:1057CB00758400D2C2C2C6D2C6C2C4D2C5C2C3304F
:1057DB00C3FD74A0F5C2C2C5C2C330C3FD8EC2C225
:1057EB00C330C3FD8FC2C2C330C3FD8DC2C2C33031
:1057FB00C3FDD2C4C2C320C4FD123633227584004C
:10580B00C2C3D2C530C3FD74A0F5C2C2C5C2C3307A
:10581B00C3FD8EC2C2C330C3FD8FC2C2C330C3FD32
:10582B00C2C4D2C5C2C330C3FD74A1F5C2C2C5C2C6
:10583B00C330C3FDC2C2C2C330C3FD85C207D2C4CD
:06584B00C2C320C4FD22CF
:08000300023C50000000000067
:08000B00023C5400000000005B
:08001300023DA90000000000FD
:0C001B00C28FB2A1320000000000000003
:09002300320000000000000000A2
:08002B00023C57000000000038
:08003300320000000000000093
:0A003B003200000000000000000089
:0900430032000000000000000082
:08004B0032000000000000007B
:08005300320000000000000073
:08005B00023CBC0000000000A3
:08006300320000000000000063
:08006B00023CD400000000007B
:08007300023C5D0000000000EA
:08007B00023DAC000000000092
:08008300023CB6000000000081
:08008B0032000000000000003B
:10009300023DCA0000000000000000000000000054
:1000A3003275FF0775FFDE75FFAD75840F75E107C8
:1000B30075E20475E34475840F75A43575A5097558
:1000C300A6FF75A7FF759CFF759D00759E00759F24
:1000D300F075D8FF75E8FF75F80F75AD0F758401DE
:1000E30075893075888F75840275893075888F7529
:1000F300840F758A80758C67780874FF0000000090
:100103000000000000000000D5E0F1D8EDE58C30E0
:10011300E7FB759701758A0043890475840075B7F9
:100123001075840F438901758D01758F01758E02DA
:100133007480D5E0FD438902E58930E4FB759702BD
:1001430075840075D10775840075BB0175BA007598
:10015300BCF075C70075C60075C5FF75C4FF75E8AB
:100163008175840275BB0475BA0075BCF175C60050
:1001730075C4FF75E88875840075D484758401752A
:10018300D484758400C2F8759A47759D1A43F8099B
:1001930075870075840075B90075A90075910075A0
:1001A300985075840175981075840075C04075C3A7
:1001B3000075CFC9758400758E1075892075880503
:1001C300758400758A00758B70758CF4758D70431A
:1001D300885075840075C90075CA0075CB0075CC4D
:1001E3000075CD0075840175C91875CA8075CBFB80
:1001F30075CDFB75CC80D2CA75840275C91875CAD2
:10020300A675CBAF75CDAF75CCA6D2CA7584007574
:10021300EF0075A8AF75B80075E6A475E71775F616
:100223000075F7019000007F007E20E4F0A3DFFC5F
:02023300DEFAF1
:10023500752EFF752FFF7530FF7531FF7532FF7510
:1002450033FF7534FF7535FF7536FF751D0A751E4D
:050255000A751F0622DE
:103C500002325E32C28D32758400C2CF32C0E0C003
:103C600083C082C0D0C000C0F0C2CFB232203223A5
:103C7000122E8C151BE51B7009751B0A75840175C6
:103C800088AF151CE51C7009751C60758402758869
:103C9000AF8011122FA2153FE53F7008753F0475E4
:103CA0008400D28B758400D2ECD0F0D000D0D0D07C
:103CB00082D083D0E032C2CF02135932C0E0C0D0EC
:103CC000E54060021540E5436002154375888FD0DA
:103CD000D0D0E032C0E0C0D0C000C084202A13752C
:103CE000840F30DF25E5E8540FF549D22A754AC81C
:103CF0008018154AE54A7006E549D2E7F54975840A
:103D00000F20DF06C22AD229D251202C1475840F2D
:103D100030F828E5E854F0C4F54BD22C754CC88037
:103D20001A154CE54C7006E54BD2E7F54B75840F40
:103D300020F808C22CD22BD250D237E541600215B0
:103D400041E55E6002155E787EE6600116151DE5B0
:103D50001D704B751D0AE54260021542E544600284
:103D60001544E55A6002155AE55B6002155B788AD6
:103D7000E6600116E55860021558E55960021559CC
:0D3D8000151EE51E7018751E0AE55D600237
:103D8D00155D151FE51F7009751F06E55C600215B1
:103D9D005CD084C28DD000D0D0D0E032021076201D
:103DAD00280DD22885BF3E85BE3D75BB01800BC257
:103DBD002885BF3C85BE3B75BB00C2ED32C0E0C05F
:103DCD00D0E54DB4000A054D85BE4875BB07803D55
:103DDD00B4010A054D85BE4575BB048030B4020A99
:103DED00054D85BE4875BB068023B4030A054D8578
:103DFD00BE4675BB048016B4040A054D85BE4875D4
:103E0D00BB058009754D0085BE4775BB04C2EDD05D
:043E1D00D0D0E032EF
:1035A60075840FD2FD2275840FC2FD2275840FD259
:1035B600FC2275840FC2FC2275840FD2FED24522EE
:1035C60075840FC245C2FE22C29322D2932275840D
:1035D6000FA2FA2275840FA2F92275840FA2DD22AA
:1035E60075840FA2DE22A2922275840FA2DA2275BA
:1035F600840FA2DB2275840FA2D82275840FA2D96C
:103606002200000000000000000000000000002270
:10361600C000C001790478B4D8FED9FAD001D00030
:1036260022C0007814123616D8FBD00022C0E075EE
:103636004005E54070FCD0E022C0E075400FE54053
:1036460070FCD0E022C0E0754064E54070FCD0E03C
:1036560022A42582F582E58335F0F58322B40A009B
:1036660022C0E0C3997001D3D0E022B506012250F2
:1036760007B5070122400122D322EF75F0648424A6
:10368600309003C1F0E5F0A375F00A842430F0A36E
:10369600E5F02430F022EF75F0648424309003C105
:0736A600F0E5F0A375F00A46
:1036AD00842430F0A3E5F02430F09003C1E0B43071
:1036BD000B7420F0A3E0B430037420F02290032D9E
:1036CD00E0540FFFA3E0B420028019540FCF75F022
:1036DD000AA42FFFA3E0B420028009540FCF75F088
:1036ED000AA42FFF22C006C005C00490032DE0548C
:1036FD000FFFFEA3E0B42003C3802C540FFDCF7544
:10370D00F00AA42FFFA3E0B42003C3801A540FFCCA
:10371D00EE75F064A420D20EFEED75F00AA42E40D5
:10372D00052C40028001D3D004D005D0062275F0BF
:10373D006484F6E5F00875F00A84F608A6F0082210
:10374D00C0017900E6B4FF028027F908E6B4FF0353
:10375D00C38022E975F00AA426F908E6B4FF03C375
:10376D008013E975F00AA420D207C3264003F9801F
:10377D0004D3D00122E9D00122E675F00AA408266F
:10378D00227850EE12373B754E00754F00785290EF
:04379D0037E7790889
:1037A100EF134007A3A3A3A3A3801CC0E0C000C0E4
:1037B10001C37905E49336D4A2E4540FF6A318D9D2
:1037C100F3D001D000D0E0D9D8E54E600C754F0997
:1037D100755009755109755209854F4E85504F85B0
:1037E10051508552512206050200000201050000D8
:1037F100040200010008040002000609000400029E
:0E380100090108000408030601080607020377
:1025710044313233343536373839302A23414243F6
:1025810044AAA3C1C2C3C4D7ABA8A92A23414243C9
:102591000101010101010101010000000000000031
:1025A100000000000000000000000000000000002A
:1025B100000000000000000000000000000000001A
:1025C100000000000000000000000000000000000A
:1025D10000000000000000000000000000000000FA
:1025E10000000000000000000000010101010101E4
:1025F10001010100000000000000000000000000D7
:1026010000000000000000000000000000000000C9
:1026110000000000000000000000000000000000B9
:1026210000000000000000000000000000000000A9
:102631000000000000000000000000000000000099
:102641000000000001010101010101010100000080
:102651000000000000000000000000000000000079
:102661000000000000000000000000000000000069
:102671000000000000000000000000000000000059
:102681000000000000000000000000000000000049
:1026910000000000000000000000000000006E06C5
:1026A100001102061501016E100611030115010149
:1026B100640116110405150101000000000000006D
:1026C1000000000000000000000000000000000009
:1026D10000000000000000000000000000000000F9
:1026E10000000000000000000000000000000000E9
:1026F10000000000000000000101010101010101D1
:1027010001000000000000000000000000000000C7
:1027110000000000000000000000000000000000B8
:1027210000000000000000000000000000000000A8
:102731000000000000000000000000000000000098
:102741000000000000000000000000000000000088
:10275100000001010101010101010100000000006F
:102761000000000000000000000000000000000068
:102771000000000000000000000000000000000058
:102781000000000000000000000000000000000048
:102791000000000000000000000000000000000038
:1027A10000000000000000000000000020202020A8
:1027B1002020202020202020202020202020202018
:1027C1002020202020202020202020202020202008
:1027D10020202020202020202020202020202020F8
:1027E10020202020202020202020202020202020E8
:1027F10020202020202020202020202020202020D8
:1028010020202020202020202020202020202020C7
:1028110020202020202020202020202020202020B7
:1028210020202020202020202020202020202020A7
:102831002020202020202020202020202020202097
:102841002020202020202020202020202020204166
:102851004E49204E554D4245522020202020202017
:10286100414E49204E414D452020202020415558C0
:102871002052454C41592056414C494420202020AA
:102881002020202020202020313D454E20202020C6
:10289100202020202020202020414E4920202020BF
:1028A1002020202020202020202020202020202027
:1028B1002020202020202020202020202020202017
:1028C100474C4F42414C202020202020204354439C
:1028D100535320434F4445202020202020204443AF
:1028E1005320434F44452020202020204C54522087
:1028F10052455045415445522020202020414E4907
:1029010020504152414D4554455253205350454565
:10291100442043414C4C494E4720202020505443F1
:10292100204E554D424552202020202020564F490F
:102931004345204D455353414745532020564F4968
:10294100434520504C41594241434B202020494EA0
:1029510056414C49442054595045202020204F5580
:1029610054204F462052414E4745202020494C4C8F
:102971004547414C2056414C554520204D55535417
:102981002046494C4C204649454C44202020494C86
:102991004C4547414C20434F44452020204441545D
:1029A1004120414343455054454420204C494E4524
:1029B100204E554D4245523A202020205553455234
:1029C1002050524F4752414D4D494E475553455264
:1029D1002049443A2020202020202020564F4943DE
:1029E10045205245434F5244494E472020494C4CC3
:1029F1004547414C20454E545259202020494C4CCA
:102A01004547414C2047414E47202020202020436C
:102A11004F4D504C4554454420202020363330360C
:102A2100373036393437313937343437373037394D
:102A31003738323538353438383539313539343835
:102A41003937343130303130333130373131303161
:102A5100313431313831323331323731333131334D
:102A6100363134313134363135313135363135392C
:102A7100313632313635313637313731313733311D
:102A810037373137393138333138363138393139EF
:102A91003231393631393932303332303632313000
:102AA10032313832323532323932333332343132F3
:102AB10035303235343030363030373031353031F1
:102AC10037303231303233303235303236303331E3
:102AD10030333230333630343330343730353030D0
:102AE10035313035333035343036353037313037B4
:102AF10032303733303734313134313135313136A9
:102B010031323231323531333131333231333431A3
:102B11003431313433313435313532313535313584
:102B2100363136323136353137323137343230356C
:102B3100323132323134323233323235323236326C
:102B4100343332343432343532343632353132354D
:102B51003232353532363132363332363532363637
:102B61003237313237343330363331313331353333
:102B7100323533333133333233343333343633351F
:102B81003133353633363433363533373134313109
:102B91003431323431333432333433313433323407
:102BA10034353434363435323435343435353436DD
:102BB10032343634343635343636353033353036D2
:102BC10035313635323335323635333235343635C3
:102BD10036353630363631323632343632373633B0
:102BE10031363332363534363632363634373033A1
:102BF1003731323732333733313733323733343792
:102C010034333735344142434445464748494A4BBA
:102C11004C4D4E4F505152535455565758595A6175
:102C210062636465666768696A6B6C6D6E6F70710B
:102C310072737475767778797A3031323334353608
:102C4100373839607E21402324255E262A28295FD2
:102C51002D2B3D7B7D5B5D7C3A3B3C3E2C2E3F2FFB
:102C610020202020202020202064010011021115A5
:102C71000101640200110311150101640400110432
:102C810011150101640800110511150101780601F2
:102C91001106011901018202071107121500638251
:102CA10002081108121500638202091109131500A7
:102CB1006382030A110A151500FF82030B110B151C
:102CC1001500FF641000110C1115051982020C1179
:102CD1000D1415016382020D110E14150063820299
:102CE1000E110F1415006382020F111013150163E9
:102CF10020202020202020202020202020202020D3
:102D010020202020202020202020202020202020C2
:102D11002054454C434F2050524F4752414D2020A3
:102D210020524144494F2050524F4752414D20209B
:102D31002050484F4E452050524F4752414D202080
:102D410020434F4D50552050524F4752414D202066
:102D5100202041434345535320434F4445202020E5
:102D6100205455524E204F4E2044454C415920206D
:102D7100205455524E204F46462044454C4159203F
:102D81005455524E2041524F554E4420444C5920E7
:102D910044544D462054454C434F204C4556454CD8
:102DA10044544D4620524144494F204C4556454CD0
:102DB10041555820524C5920494E56414C494420C6
:102DC10020494E56414C49442054494D45522020FA
:102DD100202056414C49442054494D455220202041
:102DE1002020444953504C41592054494D452020FD
:102DF100204348415241435445522054494D4520B6
:102E0100202020202020202020202020313D454E40
:102E110020202020202020202020203130204D5330
:102E210020202020202020202020313030204D5310
:102E31002020202020202020202020202053454316
:102E41002020202020202020202020524154494FA2
:102E51000F3132333435360A6314FF320505050A62
:102E61000000000000000000000000000000000061
:102E710000000000202020202020202020202020D1
:0B2E8100202020202020202020200006
:106AA600755C64E4900320F030470B30462412678F
:106AB600F5123A5980F530480B30461612683412F2
:106AC6003A5980F530490B304608123FBB123A5905
:036AD60080F52226
:103A5900E55C7012900320E0D394004009C247C28C
:103A690048C249C24622900320E01252F63B700038
:103A79003B73013B76023B79033B7C043B7E053B70
:103A890080063B82073B85083B880A3B8B0B3B8EB4
:103A99000F3B91103B94143B97153B9A193B9D1A88
:103AA9003BA01B3BA31E3BA61F3BA9233BAC243BCE
:103AB900AF283BB2293BB52D3BB82E3BBB2F3BBEB4
:103AC900303BC1323BC4333BC6343BC9353BCC6484
:103AD9003BCF653BD2663BD5673BD86E3BDA6F3B44
:103AE900DC703C1E713BDE783BE0793BE27A3C1EA0
:103AF9007B3BE4823BE6833BE8843BEA853BED8CF8
:103B09003BF08D3BF28E3BF48F3BF7963BFA973BAC
:103B1900FC983BFE993C01A03C04A13C07A23C094E
:103B2900A33C0CAA3C0EAB3C11AC3C13AD3C16B407
:103B39003C19B53C1CB63C1EB73C20BE3C23BF3CDF
:103B490026C03C29C13C1EC23C2FF03C32F13C3519
:103B5900F23C38FA3C3BFB3C3EFC3C41FD3C44FE1C
:103B69003C47FF00003C4A026F67026DC70266F5D9
:103B7900026CAA80048002800002650502412902C4
:103B89006B0C02454E0262D802469C02632A024728
:103B9900EA026777026118024D2202646C02493811
:103BA90002654F024A86026599024BD4026BCF0225
:103BB900695F0266B31265E30261748000025D7E8B
:103BC90002667002637C02662C0269D10261CE80B2
:103BD900468032804B804080228045800780268045
:103BE9003F0264B902531C801C80350263CD02591F
:103BF900548008802B0267B602549C025CA0802086
:103C09000253DC8012025AC880160243F50259D1C8
:103C1900025E58800B800C025B4102641D025694BF
:103C2900026873026282026CD1025EC1026F76027F
:103C3900622802710C02710D02710E025D0F027190
:073C49000FE4900320F022BC
:0F6F6700E4900322F0755C64900320E004F022B4
:106DC7001238FB12390A7BFF7A2979BD126B437F90
:0F6DD700111238E1C24DC24A900320E004F022AD
:1066F500304A3D900321E0FFC24ABF2A079003209C
:10670500E004F022EF642370277F231238B2900350
:1067150022E004F0E0C394034010C247C248C249D6
:10672500C246E4900320F0026E059003207402F047
:016735002241
:106CAA007BFF7A2979BD126B4312390A7F11123898
:106CBA00E112701BE490035CF07F2A1238B2C24DD5
:076CCA00900320E004F0221A
:10650500304A46900321E0F579C24AE579642A606C
:1065150038AF79126F855022AF791238B290035C8B
:10652500E02423F582E43403F583E579F090035CF8
:10653500E004F0900320E004F0227BFF7A2979ED56
:09654500126B4390032074FAF07C
:01654E00222A
:10412900204A03024293900321E0FFC24ABF2A07B3
:104139009003207403F022EF642360030242841287
:1041490038B2900324E064397077A3E06439707160
:10415900A3E06439706BD24E900323E0FFB43108B9
:10416900E4900356F00241F3EFB43208E4900357A8
:10417900F0024206EFB43302803E900323E0FFB41D
:104189003408E4900358F0024234EFB43508E4905F
:104199000359F002424AEFB43608E490035AF00298
:1041A9004260EFB437028010900323E0B4380280F4
:1041B90007900323E0B4390B7BFF7A2979FD02428A
:1041C9008AC24E900323E0FFB43016A3E0B4301145
:1041D900A3E0B4300CA3E0B43007900320740AF0D4
:1041E90022EFB4310C1260BB5007900320740FF01A
:1041F90022900323E0B4320C12605B500790032035
:104209007414F022900323E0B43311A3E0B4300C0A
:10421900126D6650079003207419F022900323E071
:10422900B4340FA3E0B4300A126EA1900320741EB7
:10423900F022900323E0B4350FA3E0B4300A126EE4
:10424900B69003207423F022900323E0B4360FA321
:10425900E0B4300A126ECB9003207428F022900348
:1042690023E0B43716A3E0B43011A3E0B4300CA3B3
:10427900E0B43007900320742DF0227BFF7A29796E
:0A428900ED126B4390032074FAF06D
:014293002208
:106B0C0090035B740BF090035C7407F0E4900369E2
:106B1C00F090036AF090036BF07BFF7A2879BD123A
:106B2C006B43126B6E7F1E1238E19003207432F0AF
:016B3C002236
:10454E00125BB6D39003C7E0940A9003C6E09400C2
:10455E00400A126B3D90032074FAF0229003C6E0DD
:10456E00FEA3E0FF902C6A75F0091252EAEE75F088
:10457E0009A42583F583E493900360F0902C6B756A
:10458E00F009EF1252EAEE75F009A42583F583E4E3
:10459E0093900361F09003C6A3E0902C6C75F00924
:1045AE001252EAEE75F009A42583F583E493900385
:1045BE0062F0902C6D75F009EF1252EAEE75F0096B
:1045CE00A42583F583E493900363F09003C6A3E0E0
:1045DE00902C6E75F0091252EAEE75F009A425833F
:1045EE00F583E493FD900364F0902C6F75F009EF62
:1045FE001252EAEE75F009A42583F583E493900335
:10460E0065F09003C6A3E0902C7075F0091252EA83
:10461E00EE75F009A42583F583E493900366F0907C
:10462E002C7175F009EF1252EAEE75F009A425838C
:10463E00F583E493900367F09003C6A3E0902C7289
:10464E0075F0091252EAEE75F009A42583F583E49C
:10465E0093900368F0ED6015900364E075F010A47C
:10466E0024F1F9742C35F0FA7BFF126B439003653D
:10467E00E0FF601175F010A424F1F9742C35F0FAF6
:0E468E007BFF126B74900360E0900320F0221B
:1062D80090035B7410F090035C7407F0E49003691A
:1062E800F090036AF0900356E090036BF07BFF7A1E
:1062F8002879CD126B43126B6E7F0D1238E1900333
:1063080024E0FF1238B2900325E0FF1238B2900360
:1063180026E0FF1238B27F1E1238E1900320743253
:02632800F02261
:10469C00125BB6D39003C7E094009003C6E094007D
:1046AC00400A126B3D90032074FAF0229003C6E08E
:1046BC00FEA3E0FF90259175F0091252EAEE75F019
:1046CC0009A42583F583E493900360F090259275FB
:1046DC00F009EF1252EAEE75F009A42583F583E494
:1046EC0093900361F09003C6A3E090259375F009B5
:1046FC001252EAEE75F009A42583F583E493900336
:10470C0062F090259475F009EF1252EAEE75F009FB
:10471C00A42583F583E493900363F09003C6A3E090
:10472C0090259575F0091252EAEE75F009A42583CF
:10473C00F583E493FD900364F090259675F009EFF2
:10474C001252EAEE75F009A42583F583E4939003E5
:10475C0065F09003C6A3E090259775F0091252EA14
:10476C00EE75F009A42583F583E493900366F0902D
:10477C00259875F009EF1252EAEE75F009A425831D
:10478C00F583E493900367F09003C6A3E09025991A
:10479C0075F0091252EAEE75F009A42583F583E44D
:1047AC0093900368F0ED6015900364E075F010A42D
:1047BC0024ADF9742735F0FA7BFF126B4390036537
:1047CC00E0FF601175F010A424ADF9742735F0FAF0
:0E47DC007BFF126B74900360E0900320F022CC
:10632A0090035B7415F090035C7407F0E4900369C2
:10633A00F090036AF0900357E090036BF07BFF7ACA
:10634A002879DD126B43126B6E7F0C1238E19003D1
:10635A0024E0FF1238B2900325E0FF1238B290030E
:10636A0026E0FF1238B27F1E1238E1900320743201
:02637A00F0220F
:1047EA00125BB6D39003C7E094009003C6E094002E
:1047FA00400A126B3D90032074FAF0229003C6E03F
:10480A00FEA3E0FF9025EB75F0091252EAEE75F06F
:10481A0009A42583F583E493900360F09025EC7551
:10482A00F009EF1252EAEE75F009A42583F583E444
:10483A0093900361F09003C6A3E09025ED75F0090B
:10484A001252EAEE75F009A42583F583E4939003E6
:10485A0062F09025EE75F009EF1252EAEE75F00952
:10486A00A42583F583E493900363F09003C6A3E041
:10487A009025EF75F0091252EAEE75F009A4258326
:10488A00F583E493FD900364F09025F075F009EF49
:10489A001252EAEE75F009A42583F583E493900396
:1048AA0065F09003C6A3E09025F175F0091252EA6B
:1048BA00EE75F009A42583F583E493900366F090DE
:1048CA0025F275F009EF1252EAEE75F009A4258374
:1048DA00F583E493900367F09003C6A3E09025F371
:1048EA0075F0091252EAEE75F009A42583F583E4FE
:1048FA0093900368F0ED6015900364E075F010A4DE
:10490A0024CDF9742735F0FA7BFF126B43900365C7
:10491A00E0FF601175F010A424CDF9742735F0FA80
:0E492A007BFF126B74900360E0900320F0227C
:106777007BFF7A2879ED126B437BFF7A2979CD125B
:106787006B747F0E1238E1900325E0FF1238B29048
:106797000326E0FF1238B27F1A1238E190035B74C8
:0F67A7001AF090035C7404F09003207432F02217
:10611800304F079003207403F022126B6E7F1E121B
:1061280038E1125F2A9003C8E0FEA3E0FFD3940091
:10613800EE9400402DEF94FBEE9400502590035B05
:10614800741BF090035C7407F0E4900369F090030B
:106158006AF0900355E01490036BF09003207432BA
:0C616800F022126B3D90032074FAF0222C
:104D2200D39003C7E094009003C6E09400400A12B7
:104D32006B3D90032074FAF0229003C6E0FEA3E0DC
:104D4200FF90264575F0091252EAEE75F009A42586
:104D520083F583E493900360F090264675F009EFA3
:104D62001252EAEE75F009A42583F583E4939003C9
:104D720061F09003C6A3E090264775F0091252EA4B
:104D8200EE75F009A42583F583E493900362F09015
:104D9200264875F009EF1252EAEE75F009A4258350
:104DA200F583E493900363F09003C6A3E090264951
:104DB20075F0091252EAEE75F009A42583F583E431
:104DC20093FD900364F090264A75F009EF1252EABF
:104DD200EE75F009A42583F583E493900365F090C2
:104DE20003C6A3E090264B75F0091252EAEE75F065
:104DF20009A42583F583E493900366F090264C750D
:104E0200F009EF1252EAEE75F009A42583F583E466
:104E120093900367F09003C6A3E090264D75F009C6
:104E22001252EAEE75F009A42583F583E493900308
:104E320068F0ED6015900364E075F010A424EDF9BC
:104E4200742735F0FA7BFF126B43900365E0FF6035
:104E52001175F010A424EDF9742735F0FA7BFF12D6
:0B4E62006B74900360E0900320F022CE
:10646C0090035B741FF090035C7407F090036974E5
:10647C0064F090036A7417F0900358E090036BF08B
:10648C007BFF7A2879FD126B43126B6E7F0F1238EB
:10649C00E1900325E0FF1238B2900326E0FF12389A
:0D64AC00B27F1E1238E19003207432F022FE
:10493800125BB6D39003C7E094039003C6E09400DB
:10494800400A126B3D90032074FAF0229003C6E0EF
:10495800FEA3E0FF90269F75F0091252EAEE75F06B
:1049680009A42583F583E493900360F09026A0754D
:10497800F009EF1252EAEE75F009A42583F583E4F5
:1049880093900361F09003C6A3E09026A175F00907
:104998001252EAEE75F009A42583F583E493900397
:1049A80062F09026A275F009EF1252EAEE75F0094E
:1049B800A42583F583E493900363F09003C6A3E0F2
:1049C8009026A375F0091252EAEE75F009A4258322
:1049D800F583E493FD900364F09026A475F009EF45
:1049E8001252EAEE75F009A42583F583E493900347
:1049F80065F09003C6A3E09026A575F0091252EA67
:104A0800EE75F009A42583F583E493900366F0908E
:104A180026A675F009EF1252EAEE75F009A425836F
:104A2800F583E493900367F09003C6A3E09026A76C
:104A380075F0091252EAEE75F009A42583F583E4AE
:104A480093900368F0ED6015900364E075F010A48E
:104A5800240DF9742835F0FA7BFF126B4390036537
:104A6800E0FF601175F010A4240DF9742835F0FAF0
:0E4A78007BFF126B74900360E0900320F0222D
:10654F0090035B7424F090035C7407F0E49003698C
:10655F00F090036AF0900359E090036BF07BFF7AA1
:10656F0029790D126B43126B6E7F0F1238E1900376
:10657F0025E0FF1238B2900326E0FF1238B27F1EDB
:0A658F001238E19003207432F0226C
:104A8600125BB6D39003C7E094009003C6E094008F
:104A9600400A126B3D90032074FAF0229003C6E0A0
:104AA600FEA3E0FF9026F975F0091252EAEE75F0C2
:104AB60009A42583F583E493900360F09026FA75A4
:104AC600F009EF1252EAEE75F009A42583F583E4A6
:104AD60093900361F09003C6A3E09026FB75F0095E
:104AE6001252EAEE75F009A42583F583E493900348
:104AF60062F09026FC75F009EF1252EAEE75F009A5
:104B0600A42583F583E493900363F09003C6A3E0A2
:104B16009026FD75F0091252EAEE75F009A4258378
:104B2600F583E493FD900364F09026FE75F009EF9B
:104B36001252EAEE75F009A42583F583E4939003F7
:104B460065F09003C6A3E09026FF75F0091252EABD
:104B5600EE75F009A42583F583E493900366F0903F
:104B6600270075F009EF1252EAEE75F009A42583C5
:104B7600F583E493900367F09003C6A3E0902701C2
:104B860075F0091252EAEE75F009A42583F583E45F
:104B960093900368F0ED6015900364E075F010A43F
:104BA600242DF9742835F0FA7BFF126B43900365C8
:104BB600E0FF601175F010A4242DF9742835F0FA81
:0E4BC6007BFF126B74900360E0900320F022DE
:1065990090035B7429F090035C7407F0E49003693D
:1065A900F090036AF090035AE090036BF07BFF7A56
:1065B90029791D126B43126B6E7F0D1238E190031E
:1065C90025E0FF1238B2900326E0FF1238B27F1E91
:0A65D9001238E19003207432F02222
:104BD400125BB6D39003C7E094009003C6E0940040
:104BE400400A126B3D90032074FAF0229003C6E051
:104BF400FEA3E0FF90275375F0091252EAEE75F018
:104C040009A42583F583E493900360F090275475F9
:104C1400F009EF1252EAEE75F009A42583F583E456
:104C240093900361F09003C6A3E090275575F009B3
:104C34001252EAEE75F009A42583F583E4939003F8
:104C440062F090275675F009EF1252EAEE75F009FA
:104C5400A42583F583E493900363F09003C6A3E053
:104C640090275775F0091252EAEE75F009A42583CE
:104C7400F583E493FD900364F090275875F009EFF1
:104C84001252EAEE75F009A42583F583E4939003A8
:104C940065F09003C6A3E090275975F0091252EA13
:104CA400EE75F009A42583F583E493900366F090F0
:104CB400275A75F009EF1252EAEE75F009A425831C
:104CC400F583E493900367F09003C6A3E090275B19
:104CD40075F0091252EAEE75F009A42583F583E410
:104CE40093900368F0ED6015900364E075F010A4F0
:104CF400249DF9742835F0FA7BFF126B4390036509
:104D0400E0FF601175F010A4249DF9742835F0FAC1
:0E4D14007BFF126B74900360E0900320F0228E
:106BCF003049079003207401F02290035B742EF07C
:106BDF0090035C7407F07BFF7A29792D126B4312B7
:0E6BEF006B6E7F1E1238E19003207432F0228C
:10695F00304F07900320742FF02290032AE0643801
:10696F006005A3E0B4390A126B3D90032074FAF06E
:10697F00227BFF7A2979DD126B4390032AE0540FB3
:09698F00F5569003207430F0224B
:1066B30090032AE064386005A3E0B4390A126B3D05
:1066C30090032074FAF0227BFF7A29793D126B4301
:1066D30090032AE0540FF556D202D20A752EFF1208
:1066E3003E217BFF7A2A790D126B4390032074FEBF
:0266F300F02293
:1065E30090032AE0540FF556304702D200123E338F
:1065F300304719202B04E54470F9123E2A7BFF7AB9
:106603002A790D126B4390032074FEF03048192051
:106613002904E54470F9123E2A7BFF7A2A790D1288
:096623006B4390032074FEF02289
:10617400304A56900321E0FF900354F0C24A12388B
:10618400B2900354E0FF126F855021900354E0FF56
:1061940090035CE02423F582E43403F583EFF0906C
:1061A400035CE004F0900320E004F022900354E048
:1061B400B42A079003207403F0227BFF7A2979ED37
:0A61C400126B4390032074FAF022DE
:105D7E00304A6A900321E0FF900354F0C24A123871
:105D8E00B2900354E0FFB42A0B90035BE090032023
:105D9E00F0D24F22EFB4230B90035BE0900320F080
:105DAE00C24F22900354E0FF126F8550219003548E
:105DBE00E0FF90035CE02423F582E43403F583EFE7
:105DCE00F090035CE004F0900320E004F0227BFFEF
:0E5DDE007A2979ED126B4390032074FAF022BB
:10667000304A3F900321E0FF900354F01238B2C239
:106680004A900354E0FFB42A0B90035BE090032090
:10669000F0D24F22EFB4230B90035BE0900320F085
:1066A000C24F227BFF7A2979ED126B43900320744D
:0366B000FAF022DB
:0A637C00900363E0FF7003304F3818
:106386001238E1126D431258088F79900361E0527A
:1063960079E57960047F3180027F301238B2304F60
:1063A60017C24FE5792430900343F09003537401EC
:0863B600F090032074F0F022C6
:0F63BE00900366E0FF1238E1900320E004F02224
:10662C00304A40900321E0FF900354F0C24A1238E4
:10663C00B2900354E0FFB42A079003207403F022B5
:10664C00126F85500F900354E090032DF0900320AF
:10665C00E004F0227BFF7A2979ED126B4390032042
:04666C0074FAF022AA
:1069D100304A32900321E0FF900354F0C24ABF2AAB
:1069E100079003207403F022900354E0B42307902E
:1069F1000320E004F0227BFF7A2979ED126B4390AA
:066A0100032074FAF022EC
:1061CE00126D439003CAEEF0A3EFF01258088F79C8
:1061DE0090035D7401F090032DE0B43108900361DB
:1061EE00E04279800E90032DE0B4301E900361E002
:1061FE00F452799003CAE0FEA3E0FFAD791257CBBB
:10620E00126EE090032074FEF0227BFF7A2979ED66
:09621E00126B4390032074FAF0A6
:016227002254
:105B4100900363E0FF7003304F561238E1126D434A
:105B51009003CAEEF0A3EFF0E4F579900361E0FF62
:105B6100E579C39F50279003CAE475F0011252D41E
:105B7100AFF0FE1258088F7A74432579F582E43428
:105B810003F583E57AF01238B2057980CE304F10F3
:105B9100C24FE57904900353F090032074F0F02292
:105BA10090035C740AF0900366E0FF1238E1900301
:045BB10020E004F0FC
:015BB50022CD
:105AC800304A75900321E0FF900354F0C24A12381F
:105AD800B2900354E0FFB42A079003207403F02225
:105AE800EFB42308900320E004F08039126F85504A
:105AF80038900354E0FF90035CE0FE04F074232E1A
:105B0800F582E43403F583EFF0900361E02409FFA4
:105B1800E433FE90035CE0D39FEE6480F8748098D1
:105B28004016900320E004F0227BFF7A2979ED12D9
:095B38006B4390032074FAF02283
:10687300304A37900321E0FF900354F0C24A1238A4
:10688300B2900354E0FFB42A079003207403F0226C
:10689300EFB42307900320E004F0227BFF7A2979E9
:0B68A300ED126B4390032074FAF0220A
:10628200126D439003CAEEF0A3EFF090035C740A20
:10629200F0E4F579900361E0FFE579C39F50279020
:1062A20003CAE475F0011252D4AFF0FE90035CE031
:1062B200FD04F074232DF582E43403F583E0FD122E
:1062C20057CB057980CE7BFF7A2A790D126B4390EA
:0562D200032074FEF042
:0162D70022A4
:105CA000304A6B900321E0FF900354F0C24A12384F
:105CB000B2900354E0FFB42A079003207403F0224B
:105CC000126F85501A900354E0FF90035CE0FE04CD
:105CD000F074232EF582E43403F583EFF080107B1B
:105CE000FF7A2979ED126B4390032074FAF0229029
:105CF0000361E02409FFE433FE90035CE0D39FEEF0
:0F5D00006480F87480984006900320E004F0223D
:10531C00900363E0FF7006204F030253C71238E17D
:10532C00126D439003CAEEF0A3EFF0125808123638
:10533C009C900361E0B401109003C3E0FF1238B2FB
:10534C009003C3E0900343F0900361E0B40220901B
:10535C0003C2E0FF1238B29003C3E0FF1238B290E0
:10536C0003C2E0900343F09003C3E0900344F09039
:10537C000361E0640370309003C1E0FF1238B29017
:10538C0003C2E0FF1238B29003C3E0FF1238B290B0
:10539C0003C1E0900343F09003C2E0900344F0900B
:1053AC0003C3E0900345F0304F11C24F900361E00E
:1053BC00900353F090032074F0F022900366E0FF0A
:1053CC001238E190035C740AF0900320E004F022A0
:1064B9001236F25002803B1236CA8F79900367E098
:1064C900FFE579C39F402B900368E0FFE579D39FEF
:1064D9005020126D439003CAEEF0A3EFF0AD79128C
:1064E90057CB7BFF7A2A790D126B4390032074FEF8
:0B64F900F022126B3D90032074FAF0BB
:016504002274
:1063CD001236F25002803F1236CA8F79900367E081
:1063DD00FFE579C39F400B900368E0FFE579D39FFC
:1063ED004004E5797020126D439003CAEEF0A3EFDF
:1063FD00F0AD791257CB7BFF7A2A790D126B439052
:0F640D00032074FEF022126B3D90032074FAF00E
:01641C00225D
:10595400900363E0FF7003304F5E1238E1126D4331
:105964009003CAEEF0A3EFF01258088F7912585141
:10597400E4F57974C12579F582E43403F583E0FF15
:1059840074432579F582E43403F583EFF074C1257B
:1059940079F582E43403F583E0FF1238B20579E542
:1059A40079C3940440CD304F0FC24F900353740316
:1059B400F090032074F0F022900366E0FF1238E1C7
:0C59C40090035C740AF0900320E004F0F3
:0159D00022B4
:1067B6007F0A12507B8F79E5796012126D43900340
:1067C600CAEEF0A3EFF0E57914FD1257CBE5797B1D
:1067D600FF600E7A2A790D126B4390032074FEF047
:0E67E600227A29798D126B4390032074FAF009
:0167F4002282
:10549C00900363E0FF7006204F030255371238E18A
:1054AC00126D439003CAEEF0A3EFF01258081236B7
:1054BC009C9003CAE475F0011252D4AFF0FE12585E
:1054CC00081236809003C2E0FF900343F0A3F01261
:1054DC0038B29003C3E0FF1238B29003CAE475F0FF
:1054EC00011252D4AFF0FE1258081236809003C14C
:1054FC00E0FF900345F09003C2E0900346F0900368
:10550C00C3E0900347F01238B29003C2E0FF1238A8
:10551C00B29003C3E0FF1238B2304F0FC24F90036A
:10552C00537405F090032074F0F022900366E0FFB2
:10553C001238E190035C740AF0900320E004F0222E
:1053DC0090032DE0540F75F00AA4FFA3E0540F2F97
:1053EC00F579900330E0540F75F00AA4FDACF09001
:1053FC00032FE0540F75F064A42DFFE5F03CFE90F4
:10540C000331E0540F7C002FFFEC3EFEE579C39492
:10541C00014019E579D394145012C3EF9401EE9422
:10542C00004009D3EF94FAEE9400400A126B3D90C1
:10543C00032074FAF022126D439003CAEEF0A3EF2E
:10544C00F09003CAE475F0011252D4AFF0FEAD79BE
:10545C001257CB900330E0540F75F00AA4FF900361
:10546C002FE0540F75F064A42FFF900331E0540F1C
:10547C002FF5799003CAE0FEA3E0FFAD791257CB6C
:0F548C007BFF7A2A790D126B4390032074FEF098
:01549B0022EE
:1043F5007F0D12507BEF701A900330E0B43010A39C
:10440500E0B4300BA3E0B43006A3E06430600302EF
:1044150044EE900334E0FF64306004EFB4350E9051
:104425000335E0540FD3940540030244EE90033462
:10443500E0FF64316004EFB43611900339E0B42035
:1044450007900338E0B420030244EE900334E0FF04
:1044550064326004EFB43711900338E0B42007905C
:104465000337E0B420030244EE900334E0FF6433E5
:104475006004EFB43809900335E0B42002806A90F7
:104485000334E0FF64346005EF64397066900335EA
:10449500E0540F75F00AA4FFA3E0540F2FF57990AF
:1044A5000338E0540F75F00AA4FDACF0900337E033
:1044B500540F75F064A42DFFE5F03CFE900339E040
:1044C500540F7C002FFFEC3EFEE579C394014019A3
:1044D500E579D394145012C3EF9401EE940040098A
:1044E500D3EF94FAEE9400400A126B3D90032074CA
:1044F500FAF022126D439003CAEEF0A3EFF0900399
:104505005C740AF0E4F579900361E0FFE579C39FF7
:1045150050279003CAE475F0011252D4AFF0FE9013
:10452500035CE0FD04F074232DF582E43403F58388
:10453500E0FD1257CB057980CE7BFF7A2A790D12E3
:084545006B4390032074FEF0AB
:01454D00224B
:1059D100900363E0FF7003304F5B1238E1126D43B7
:1059E1009003CAEEF0A3EFF0E4F579900361E0FFD4
:1059F100E579C39F502C9003CAE475F0011252D48B
:105A0100AFF0FE1258088F7A74432579F582E43499
:105A110003F583E57AF07E001258081238B2057951
:105A210080C9304F10C24FE57904900353F09003C1
:105A31002074F0F022900366E0FF1238E190035CDD
:0B5A4100740AF0D24D900320E004F046
:015A4C002237
:105E5800304A65900321E0FF900354F0C24ABF2AFC
:105E6800079003207403F022900354E0FFB4230842
:105E7800900320E004F0803DEF547FFF1238B29089
:105E88000354E0547FFF90035CE0FE04F074232E7B
:105E9800F582E43403F583EFF0900361E02409FF11
:105EA800E433FE90035CE0D39FEE6480F87480983E
:095EB8004006900320E004F022F2
:10641D00304A4B900321E0FF900354F0C24ABF2A4B
:10642D00079003207403F022900354E0FFB4230B74
:10643D00900320E004F0E004F08010126F85500FFF
:10644D00900354E090035EF0900320E004F0227B73
:0F645D00FF7A2979ED126B4390032074FAF02235
:10569400204A03025730900321E0FF900354F0C2E4
:1056A4004ABF2A079003207403F022900354E0FFBA
:1056B400B4230A900320E004F0E004F022126F8582
:1056C400505B90035EE0540F75F00AA4FF900354FE
:1056D400E0540F2FF0E0902C0693FF900354F01247
:1056E40038B2900354E0FF90035CE0FE04F07423AE
:1056F4002EF582E43403F583EFF0900361E024098E
:10570400FFE433FE90035CE0D39FEE6480F8748082
:1057140098900320E0400304F02214F0227BFF7AE7
:0D5724002979ED126B4390032074FAF022F6
:106CD1003047099003D5E0F55B1235A6304903E44E
:106CE100F55B30480B304505755B0A8003755B2801
:076CF100900320E004F022F3
:105EC100E55B7064125169900360E01252F65EF175
:105ED100645EF66E5EF6785EF6825EF68C5EFB962A
:105EE1005F00A05F05AA5F0AB45F0FBE00005F12EA
:105EF100126E74801C126B9F801712711080121227
:105F01007111800D127112800812711380031271C8
:105F11001430470E9003D4E0787EF6900320E0041D
:095F2100F0229003207401F0222B
:0F6F7600787EE670091235AC9003207401F0228A
:1062280030470D9003D5E0F55B1235A6E55B70FCB1
:10623800304807755B05E55B70FCE4F57930480C80
:1062480012706F12364B1270F812364B30470C1220
:10625800707A12364B1270F812364B0579E579C30D
:10626800940540D930470C9003D4E0787EF6787EC8
:09627800E670FB9003207401F0B4
:0162810022FA
:01710C002260
:01710D00225F
:01710E00225E
:105D0F0030480A2045079003207401F02230470DD8
:105D1F009003D5E0F55B1235A6E55B70FC304807C4
:105D2F00755B05E55B70FC30471512707AE4F57909
:105D3F0012364B0579E579C3940A40F41270F830A6
:105D4F00481512706FE4F57912364B0579E579C372
:105D5F00940A40F41270F830470C9003D4E0787E28
:0E5D6F00F6787EE670FB126E05E4900320F0DD
:015D7D002203
:01710F00225D
:1067F500302B3B204A38755C64E54B547FFF902570
:106805007193900321F0304D0EE54B30E709EF9081
:10681500258193900321F0D24AC22B900321E0B445
:0F6825002307900322E004F022E4900322F022E4
:1068340030293B204A38755C64E549547FFF902534
:106844007193900321F0304D0EE54930E709EF9044
:10685400258193900321F0D24AC229900321E0B408
:0F6864002307900322E004F022E4900322F022A5
:103FBB00204B03024128304A03024128900322E0A0
:103FCB00F579E4F0755C64127106D24ABF30079044
:103FDB0003217430F022BF31079003217431F0229A
:103FEB00BF32079003217432F022BF3307900321B5
:103FFB007433F022BF34079003217434F022BF35A1
:10400B00079003217435F022BF36079003217436D5
:10401B00F022BF37079003217437F022BF38079087
:10402B0003217438F022BF39079003217439F02231
:10403B00BF23109003217423F0AF790579900322ED
:10404B00EFF022BF2A07900321742AF022BF410709
:10405B009003217441F022BF42079003217442F078
:10406B0022BF43079003217443F022BF64079003E0
:10407B00217444F022204D03C24A22BF61079003F2
:10408B00217461F022BF62079003217462F022BF9A
:10409B0063079003217463F022BF640790032174BC
:1040AB0064F022BF65079003217465F022BF660799
:1040BB009003217466F022BF67079003217467F0A9
:1040CB0022BF68079003217468F022BF6907900331
:1040DB00217469F022BF6A07900321746AF022BF32
:1040EB006B07900321746BF022BF6C079003217454
:1040FB006CF022BF6D07900321746DF022BF6E0729
:10410B00900321746EF022BF6F07900321746FF040
:0D411B0022BF70079003217470F022C24A89
:014128002274
:0B701B007F209003237420F0A3DFFC13
:017026002247
:0F6F8500EFC394304007EFD39439500122C32259
:105BB60090032CE0FD6420602E90032BE0540F75BB
:105BC600F00AA4FBAAF090032AE0540F75F064A42F
:105BD6002BFFE5F03AFEED540F7C002FFFEC3E90D4
:105BE60003C6F0A3EF803190032BE0FD6420900301
:105BF6002A601AE0540F75F00AA4FFED540F7C00DA
:105C06002FFEEC35F09003C6F0A3CE800BE0540FC8
:105C1600FF9003C6E4F0A3EFF0E024FFF09003C684
:055C2600E034FFF02254
:105F2A00900329E0FD6420602B900328E0540F754C
:105F3A00F00AA4FBAAF0900327E0540F75F064A4BA
:105F4A002BFFE5F03AFEED540F7C002FFFEC3E905C
:105F5A0003C8802E900328E0FD6420900327601A6E
:105F6A00E0540F75F00AA4FFED540F7C002FFEECED
:105F7A0035F09003C8F0A3CEF022E0540FFF90034F
:075F8A00C8E4F0A3EFF022D0
:106D6600900325E0540F75F00AA4FFA3E0540F2FFB
:106D7600900355F0D394004006E09415500122C3C9
:016D860022EA
:1060BB00E4FFEF75F003A4241DF582E4342AF58385
:1060CB00E493FE900324E0FDEE6D703BEF75F0035F
:1060DB00A4241EF582E4342AF583E493FE90032571
:1060EB00E0FDEEB50521EF75F003A4241FF582E466
:1060FB00342AF583E493FE900326E0FDEEB5050705
:0C610B00900356EFF0D3220FBF33A7C360
:016117002265
:10605B00E4FF75F003EFA424B6F582E5F0342AF5DE
:10606B0083E493FE900324E0FDEE6D703D75F00329
:10607B00EFA424B7F582E5F0342AF583E493FE9080
:10608B000325E0FDEEB5052275F003EFA424B8F56A
:10609B0082E5F0342AF583E493FE900326E0FDEECF
:0F60AB00B50507900357EFF0D3220FBF70A4C3C2
:0160BA0022C3
:10507B0074232FF582E43403F583E0FD643170690A
:10508B00FE74242FF582E43403F583E0FCEE75F017
:10509B0003A4241DF582E4342AF583E4936C704257
:1050AB0074252FF582E43403F583E0FCEE75F003F1
:1050BB00A4241EF582E4342AF583E493B504237407
:1050CB00262FF582E43403F583E0FCEE75F003A4A0
:1050DB00241FF582E4342AF583E493B50404EE042B
:1050EB00FF220EBE339B7F0022ED6432706DFE7487
:1050FB00242FF582E43403F583E0FD75F003EEA471
:10510B0024B6F582E5F0342AF583E4936D7045748B
:10511B00252FF582E43403F583E0FD75F003EEA44F
:10512B0024B7F582E5F0342AF583E493B5052574AD
:10513B00262FF582E43403F583E0FD75F003EEA42E
:10514B0024B8F582E5F0342AF583E493B50505EE32
:0D515B002434FF220EBE70977F00227F00DB
:015168002224
:10585100EFC394339003C150397431F0EF75F00305
:10586100A4241DF582E4342AF583E4939003C2F065
:10587100EF75F003A4241EF582E4342AF583E49342
:105881009003C3F0EF75F003A4241FF582E4342ADA
:10589100803A7432F075F003EFA4241DF582E5F02F
:1058A100342AF583E4939003C2F075F003EFA42446
:1058B1001EF582E5F0342AF583E4939003C3F07575
:1058C100F003EFA4241FF582E5F0342AF583E49375
:0558D1009003C4F02269
:106EA100900325E0540F75F00AA4FFA3E0540F2FBF
:056EB100900358F022DF
:106EB600900325E0540F75F00AA4FFA3E0540F2FAA
:056EC600900359F022C9
:106ECB00900325E0540F75F00AA4FFA3E0540F2F95
:056EDB0090035AF022B3
:066B3D007BFF7A29795D5F
:066B43008B7A8A7B897C3D
:106B49007F011238E1E4F57DAB7AAA7BA97C857DCA
:106B590082758300125252FF1238B2057DE57DC35A
:046B6900941040E460
:016B6D002205
:066B6E007BFF7A2979ADDE
:066B74008B7A8A7B897C0C
:106B7A007F111238E1E4F57DAB7AAA7BA97C857D89
:106B8A0082758300125252FF1238B2057DE57DC329
:046B9A00941040E42F
:016B9E0022D4
:106D430090036BE0FF90036AE08FF0A4FF90036968
:106D5300E07C002FFFEC35F0FE900362E02FFFECA8
:036D63003EFE22CF
:106EE000900364E075F010A424F1F9742C35F0FAE5
:056EF0007BFF026B7442
:037106007F0322E2
:106E4100E4F579AF797E00E579902E5193FD1257E3
:0A6E5100CB0579E579C3941040E900
:016E5B002214
:10699800E4F579E4F57AE57975F017A42464FFE461
:1069A80035F0FE7C00EF257AFFEC3EFEE57A902E6E
:1069B8007593FD1257CB057AE57AC3941740D7052E
:0869C80079E579C3946440CB2A
:0169D00022A4
:106CF800E4F579AF797E0012580874CC2579F582CD
:106D0800E43403F583EFF00579E579C3941040E3A3
:066D18009003CCE0F5241D
:016D1E002252
:106E7400304708900343E0FF127033304808900312
:076E840043E0FF127027221A
:106B9F00E4F579900353E0FFE579C39F50217443E7
:106BAF002579F582E43403F583E0F57A304704FF65
:0F6BBF00127033304805AF7A127027057980D4F1
:016BCE0022A4
:01711000225C
:01711100225B
:01711200225A
:017113002259
:017114002258
:0C7027001270E812364B1270FF02364B5C
:0C7033001270F012364B1270FF02364B48
:10516900E4F579F57AF57B9003C7E02401FF900314
:10517900C6E03400FEC3EF940AEE94005005A3E0A4
:1051890004F57BD3EF9463EE9400404C9003C7E0A1
:105199002401FB9003C6E03400FA7C007D64AF0370
:1051A900FE12527F8F79EF75F064A4FFC3EB9FFF66
:1051B900EA95F0FE7C007D0A12527F8F7AA3E00403
:1051C900FFE57975F064A4FEC3EF9EFFE57A75F0FB
:1051D9000AA4FEC3EF9EF57B9003C7E02401FF906C
:1051E90003C6E03400FED3EF9409EE940040197C25
:1051F900007D0A12527F8F7AA3E004FFE57A75F0E9
:105209000AA4FEC3EF9EF57B74302579F5797430D5
:10521900257AF57A7430257BF57B304714AF7912FE
:105229007033AF7A127033AF7B1270337F2A1270EA
:1052390033304814AF79127027AF7A127027AF7BD9
:085249001270277F2A12702762
:01525100223A
:106D1F002A2A3132333435362A2A2A2A3132333469
:106D2F0035302A2A44313233343536373839302A20
:046D3F002341424367
:10554C00305023C250E54B540F906D33939003EEC3
:10555C00F0788A76329003DFE004F0302115126A7D
:10556C003C1268E9800D788AE670089003DAF090B6
:10557C0003EBF030513DC251E549540F906D33931C
:10558C009003EDF0125FF77558329003DFE004F0F2
:10559C003045032020062045063022031268AE3029
:1055AC004503202003204503126A07204511126A87
:1055BC00D9800CE55870089003DBF09003EAF030CA
:1055CC004C19302322125FF775593212710990036E
:1055DC00DEEFF0C24C126924026A71E55970089032
:0855EC0003DCF09003ECF02257
:106A07009003DBE0FF04F0EF906D1F93FF9003ED21
:106A1700E0FEEF6E6011EEB42A089003DB7401F01C
:106A27008005E49003DBF09003DBE0B40A06E4F0B2
:056A3700D248D25222FA
:106A3C009003DAE0FF04F0EF906D1F93FF9003EEEC
:106A4C00E0FEEF6E6011EEB42A089003DA7401F0E8
:106A5C008005E49003DAF09003DAE0B40A06E4F07F
:056A6C00D247D25222C6
:106A71009003DCE0FF04F0EF906D1F93FF9003DEC5
:106A8100E0FEEF6E6011EEB42A089003DC7401F0B1
:106A91008005E49003DCF09003DCE0B40A06E4F046
:056AA100D249D252228F
:1068AE009003EAE0FF04F074E12FF582E43403F57F
:1068BE0083E0FF9003EDE0FEEF6E6011EEB423086F
:1068CE009003EA7401F08005E49003EAF09003EA85
:0B68DE00E0B40906E4F0D248D24622E4
:1068E9009003EBE0FF04F074E12FF582E43403F543
:1068F90083E0FF9003EEE0FEEF6E6011EEB4230833
:106909009003EB7401F08005E49003EBF09003EB46
:0B691900E0B40906E4F0D247D24622A9
:106924009003ECE0FF04F074E12FF582E43403F506
:1069340083E0FF9003DEE0FEEF6E6011EEB4230807
:106944009003EC7401F08005E49003ECF09003EC08
:0B695400E0B40906E4F0D249D246226C
:106AD9009003DDE0FF04F0EF906D2993FF9003ED43
:106AE900E0FEEF6E6011EEB42A089003DD7401F048
:106AF9008005E49003DDF09003DDE0B40A04E4F0DE
:036B0900D2532242
:106BFD009003E17423F0A3F0E4FF74CD2FF582E44C
:106C0D003403F583E0FE74E32FF582E43403F5835A
:0C6C1D00EEF00FBF06E49003E97423F0D2
:016C29002248
:106E050012380F1238FB12390A7F011238E1E4906B
:0D6E150003DFF07F109003B1E4F0A3DFFC79
:016E2200224D
:105FF7009003DFE0FED3940F50129003EDE0FF749F
:10600700B12EF582E43403F583EF80437F01123824
:10601700E1E4F57974B22579F582E43403F583E098
:10602700FF74B12579F582E43403F583EFF074B199
:106037002579F582E43403F583E0FF1238B2057958
:10604700E579C3940F40CD9003EDE0FF9003C0F0D6
:036057001238B24A
:01605A002223
:037109007F0122E1
:103E2100755500123E3C50FB22755500123EC5509F
:103E3100FB22755500123E7C50FB22758400E5552E
:103E410075F003A4903E4973023EE1023EF0023F49
:103E51000E023EF7023F1A023F21023F29023EF0C5
:103E6100023F37023EF7023F47023F50023EE10266
:103E71003EF0023F5E023EF7023F6A758400E5555F
:103E810075F003A4903E8973023EE1023EF0023FC9
:103E91000E023EF7023F1A023F21023EE1023EF0CE
:103EA100023F0E023EF7023F1A023F21023F1A0271
:103EB1003F21023F29023EF0023F6C023EF7023FE2
:103EC10047023F6A758400E55575F003A4903ED220
:103ED10073023EE1023EF0023F5E023EF7023F6A9C
:103EE100C2FA123F7C123F7C759B000555C32230FC
:103EF100F9020555C32230F912E59A20E7FB123F7A
:103F01007CD2FA123F7C123F7C0555C322C2FA12C1
:103F11003F7C759B040555C32275431E0555C3227D
:103F2100E54370020555C322C2FA123F7C123F9D40
:103F3100F59B0555C322C2FA123F7C123FAC4407E0
:103F4100F59B0555C322123F8EF5440555C32275D5
:103F5100840F30DE04E54470020555C322C2FA1213
:103F61003F7C759B080555C322D322C2FA123F7CC0
:093F7100123FAC4405F59B055517
:103F7A00C322000000000000000000000000000052
:103F8A0000000022903F95E55693225A5A5A5A5AEF
:103F9A00FAFAFA903FA4E556932200B45AE12D8723
:103FAA007ADB903FB3E556932200000000000080C0
:013FBA008086
:101B310043544353532036332E302020202020207D
:101B410043544353532036372E3020202020202069
:101B510043544353532036392E3420202020202053
:101B610043544353532037312E3920202020202045
:101B710043544353532037342E3420202020202037
:101B810043544353532037372E3020202020202028
:101B910043544353532037392E372020202020200F
:101BA10043544353532038322E3520202020202007
:101BB10043544353532038352E34202020202020F5
:101BC10043544353532038382E35202020202020E1
:101BD10043544353532039312E35202020202020D7
:101BE10043544353532039342E38202020202020C1
:101BF10043544353532039372E34202020202020B2
:101C01004354435353203130302E302020202020A4
:101C11004354435353203130332E3520202020208C
:101C21004354435353203130372E3220202020207B
:101C31004354435353203131302E3920202020206A
:101C41004354435353203131342E38202020202057
:101C51004354435353203131382E38202020202043
:101C61004354435353203132332E3020202020203F
:101C71004354435353203132372E33202020202028
:101C81004354435353203133312E38202020202018
:101C91004354435353203133362E35202020202006
:101CA1004354435353203134312E332020202020FC
:101CB1004354435353203134362E322020202020E8
:101CC1004354435353203135312E342020202020DA
:101CD1004354435353203135362E372020202020C2
:101CE1004354435353203135392E382020202020AE
:101CF1004354435353203136322E322020202020AA
:101D01004354435353203136352E35202020202093
:101D11004354435353203136372E3920202020207D
:101D21004354435353203137312E33202020202078
:101D31004354435353203137332E38202020202061
:101D41004354435353203137372E33202020202052
:101D51004354435353203137392E3920202020203A
:101D61004354435353203138332E35202020202033
:101D71004354435353203138362E32202020202023
:101D81004354435353203138392E39202020202009
:101D91004354435353203139322E38202020202000
:101DA1004354435353203139362E362020202020EE
:101DB1004354435353203139392E352020202020DC
:101DC1004354435353203230332E352020202020DA
:101DD1004354435353203230362E352020202020C7
:101DE1004354435353203231302E372020202020BA
:101DF1004354435353203231382E312020202020A8
:101E01004354435353203232352E37202020202093
:101E11004354435353203232392E31202020202085
:101E21004354435353203233332E36202020202075
:101E31004354435353203234312E38202020202064
:101E41004354435353203235302E33202020202059
:101E51004354435353203235342E31202020202047
:101E61002020202020202020202020202020202071
:101E71004443532030303620494E562030323120F1
:101E81004443532030303720494E562032313420DC
:101E91004443532030313520494E562031343120CE
:101EA1004443532030313720494E562030353020BD
:101EB1004443532030323120494E562030303620B1
:101EC1004443532030323320494E5620303437209A
:101ED1004443532030323520494E56203234342089
:101EE1004443532030323620494E56203436342074
:101EF1004443532030333120494E56203632372067
:101F01004443532030333220494E5620303531205E
:101F11004443532030333620494E56203137322046
:101F21004443532030343320494E56203434352035
:101F31004443532030343720494E56203032332029
:101F41004443532030353020494E5620303137201C
:101F51004443532030353120494E5620303332200E
:101F61004443532030353320494E562034353220F6
:101F71004443532030353420494E562034313320E8
:101F81004443532030363520494E562032373120D4
:101F91004443532030373120494E562033303620C8
:101FA1004443532030373220494E562032343520B5
:101FB1004443532030373320494E562035303620A4
:101FC1004443532030373420494E56203137342092
:101FD1004443532031313420494E56203731322089
:101FE1004443532031313520494E5620313532207A
:101FF1004443532031313620494E56203735342061
:102001004443532031323220494E5620323235205A
:102011004443532031323520494E56203336352042
:102021004443532031333120494E56203336342036
:102031004443532031333220494E56203534362023
:102041004443532031333420494E56203232332019
:102051004443532031343120494E5620303135200C
:102061004443532031343320494E562034313220F9
:102071004443532031343520494E562032373420E1
:102081004443532031353220494E562031313520D9
:102091004443532031353520494E562037333120C2
:1020A1004443532031353620494E562032363520AF
:1020B1004443532031363220494E562035303320A7
:1020C1004443532031363520494E56203235312094
:1020D1004443532031373220494E56203033362085
:1020E1004443532031373420494E56203037342071
:1020F1004443532032303520494E56203236332066
:102101004443532032313220494E56203335362054
:102111004443532032313420494E56203030372049
:102121004443532032323320494E56203133342038
:102131004443532032323520494E56203132322029
:102141004443532032323620494E56203431312017
:102151004443532032343320494E56203335312005
:102161004443532032343420494E562030323520F6
:102171004443532032343520494E562030373220E3
:102181004443532032343620494E562035323320D1
:102191004443532032353120494E562031363520C3
:1021A1004443532032353220494E562034363220B2
:1021B1004443532032353520494E5620343436209D
:1021C1004443532032363120494E56203733322092
:1021D1004443532032363320494E56203230352085
:1021E1004443532032363520494E5620313536206E
:1021F1004443532032363620494E5620343534205C
:102201004443532032373120494E56203036352051
:102211004443532032373420494E5620313435203F
:102221004443532033303620494E56203037312035
:102231004443532033313120494E56203636342021
:102241004443532033313520494E56203432332014
:102251004443532033323520494E562035323620FF
:102261004443532033333120494E562034363520F0
:102271004443532033333220494E562034353520E0
:102281004443532033343320494E562035333220D2
:102291004443532033343620494E562036313220C0
:1022A1004443532033353120494E562032343320B4
:1022B1004443532033353620494E562032313220A3
:1022C1004443532033363420494E56203133312094
:1022D1004443532033363520494E56203132352080
:1022E1004443532033373120494E5620373334206D
:1022F1004443532034313120494E56203232362066
:102301004443532034313220494E56203134332056
:102311004443532034313320494E56203035342044
:102321004443532034323320494E56203331352033
:102331004443532034333120494E56203732332021
:102341004443532034333220494E56203531362010
:102351004443532034343520494E56203034332001
:102361004443532034343620494E562032353520EB
:102371004443532034353220494E562030353320E2
:102381004443532034353420494E562032363620CA
:102391004443532034353520494E562033333220BF
:1023A1004443532034363220494E562032353220B0
:1023B1004443532034363420494E5620303236209F
:1023C1004443532034363520494E5620333331208F
:1023D1004443532034363620494E56203636322077
:1023E1004443532035303320494E56203136322074
:1023F1004443532035303620494E56203037332060
:102401004443532035313620494E5620343332204F
:102411004443532035323320494E5620323436203E
:102421004443532035323620494E5620333235202D
:102431004443532035333220494E56203334332020
:102441004443532035343620494E5620313332200F
:102451004443532035363520494E562037303320FA
:102461004443532036303620494E562036333120EE
:102471004443532036313220494E562033343620DE
:102481004443532036323420494E562036333220CD
:102491004443532036323720494E562030333120C1
:1024A1004443532036333120494E562036303620AE
:1024B1004443532036333220494E5620363234209D
:1024C1004443532036353420494E56203734332087
:1024D1004443532036363220494E56203436362076
:1024E1004443532036363420494E5620333131206F
:1024F1004443532037303320494E5620353635205A
:102501004443532037313220494E56203131342053
:102511004443532037323320494E5620343331203F
:102521004443532037333120494E5620313535202D
:102531004443532037333220494E5620323631201E
:102541004443532037333420494E5620333731200A
:102551004443532037343320494E562036353420F6
:102561004443532037353420494E562031313620EB
:104F750075840F1200A4126BFD126E05126E23E4E8
:104F85009003F3F0A3F09003F1F0A3F07890F67896
:104F95008EF67892F67895F6788BF6788CF6788D8D
:104FA500F61232BB123355125DEC1270DFE542701A
:104FB500031238FB30362D1233887893E6B5071B7C
:104FC500788B06E6B41410D25A1233887893A60764
:104FD50075421EE4788BF6C23680091233887893C1
:104FE500A607C236303310788D06E6B41407D25BB7
:104FF50075421EE4F6C233305610788C06E6B408C6
:1050050007D25C75421EE4F6C256305A03125F9110
:10501500305B03125C2B305C031255F412554C3097
:105025005305125A4DC25330522FC2527F0C1239BA
:1050350028126E41126998126CF8126BFDE4900308
:10504500D9F0C247C248C249F57812364B0578E512
:1050550078C3941E40F4126E05204603024FA61233
:105065006AA6126CF8126BFDE49003D9F0C247C230
:0650750048C249024FA6EB
:104E6D0009920A9E0BC70D100E7D101211D213C59B
:104E7D0015ED185208D0094E09D40A600AF40B91A9
:104E8D000C360CE50D9D0E600F2D100610EB11DD8F
:104E9D0012DC13EA15071633177118C01D2107B15F
:104EAD0007E808200859196E1A211ADA1B971C5A9F
:104EBD000894090E09900A190AA90B410BE30C8CF1
:104ECD000D3F0DFD0EC50F9810771162125B136229
:104EDD001477159B16D018161DEF1EC21F9B207937
:104EED00215F224A233B24342533263912330FCD3B
:104EFD0014331566169A17CD19000E9A1366110004
:104F0D0011661033150016331766189A19CD0DCD8D
:104F1D000F00129A11CD1300149A15CD17001833E6
:104F2D0019660E330F66109A191823A01296203D9C
:104F3D00129623A0129627631488203D148823A06F
:104F4D001488276316B8203D16B823A016B827631A
:104F5D001918203D1918276312962B8C14882B8C49
:084F6D0016B82B8C19182B8CCF
:0B706F0075081575095ED22DD20322B2
:0B707A0075081575095ED22DD20B229F
:0770F800C22DC203C20B22EE
:0870E800124294D22ED20422C0
:0870F000124294D22ED20C22B0
:09429400E4F512F513F514F5151B
:10429D00EF1252F643982343872A42D53042E73135
:1042AD0042F932430B33431D34432F3543413643DB
:1042BD00533743653843763943A94143BA4243CB1B
:1042CD004343DC44000043F4904F35E493F50D7403
:1042DD000193F50E904F370243EB904F39E493F570
:1042ED000D740193F50E904F3B0243EB904F3DE45F
:1042FD0093F50D740193F50E904F3F0243EB904FE4
:10430D0041E493F50D740193F50E904F430243EB89
:10431D00904F45E493F50D740193F50E904F4702C0
:10432D0043EB904F49E493F50D740193F50E904FC7
:10433D004B0243EB904F4DE493F50D740193F50E45
:10434D00904F4F0243EB904F51E493F50D74019351
:10435D00F50E904F530243EB904F55E493F50D74CA
:10436D000193F50E904F578075904F59E493F50DCD
:10437D00740193F50E904F5B8064904F5DE493F55F
:10438D000D740193F50E904F5F8053904F61E49340
:10439D00F50D740193F50E904F638042904F65E4D7
:1043AD0093F50D740193F50E904F678031904F6921
:1043BD00E493F50D740193F50E904F6B8020904FA3
:1043CD006DE493F50D740193F50E904F6F800F9082
:1043DD004F71E493F50D740193F50E904F73E493C3
:0843ED00F50F740193F5102295
:0770FF00C22EC20CC20422E4
:10107600C0D0C000C001C083C082C0E0C0F0A29250
:1010860020A001B37884E233F208E233F208E233B7
:10109600F208E233F208E233F208E233F208E2330E
:1010A600F208E233F208E233F208E233F208E233FE
:1010B600F208E233F208E233F208E233F208E233EE
:1010C600F208E233F208E233F208E233F208E233DE
:1010D600F208E233F208E233F208E233F208E233CE
:1010E600F208E233F208E233F208E233F208E233BE
:1010F600F208E233F208E233F208E233F208E233AE
:10110600F208E233F208E233F208E233F208E2339D
:10111600F208E233F208E233F208E233F208E2338D
:10112600F208E233F29014E178ABE218936028E219
:1011360018937023E21893601EE218937019E21850
:10114600936014E21893600FE21893700AE2189302
:101156007005E21893600302130B756000E21893A2
:101166001392545003756038752300E21893139256
:101176001C500363601CE2189313921B50036360B8
:101186000EE2189313921A5003636046E218931303
:1011960092195003636023E2189313921885236112
:1011A6005003636051752300E2189313921C500399
:1011B600636068E2189313921B5003636075E2182C
:1011C6009313921A500363607AE21893139219509C
:1011D6000363603DE21893139218852362500363FC
:1011E600601F752300E2189313921F500363604F2C
:1011F600E2189313921E5003636026E2189313922B
:101206001D5003636052E2189313921C50036360EF
:1012160029E2189313921B5003636015E218931387
:10122600921A500363600BE21893139219500363EA
:101236006045E21893139218852363500363606236
:10124600E2189313921C5003636031E218931392D1
:101256001B5003636019E2189313921A50036360DC
:101266000DE218931392195003636007E218931363
:1012760092188523645003636043752300E2189334
:1012860013921EE2189313921DE2189313921CE216
:10129600189313921BE2189313921AE2189313925F
:1012A60019E21893139218852365C257E5656560A0
:1012B6006035D25723F8901A3293F9901A31E89391
:1012C6006025B40104B254801EB40205E862618050
:0D12D60016B40305E86262800EB40405E85A
:1012E30062638006B40521E86264A25492559003B8
:1012F300ACE561F09003ADE562F09003AEE563F019
:101303009003AFE564F0D25612131DD0F0D0E0D0B5
:1013130082D083D001D000D0D0327880E6603630DE
:101323003133787FE6D5E02D76087880167885E628
:10133300A2E0304301B39241D23EA2E07881E613AA
:10134300F67882E613F67883E613F67884E613F6E6
:101353007885E613F622C0D0C000C001C083C082E6
:10136300C0E0C0F0C258A292205801B3786CE213D7
:10137300F208E213F208E213F208E213F208E213AE
:10138300F208E213F208E213F208E213F208E2139E
:10139300F208E213F208E213F208E213F208E2138E
:1013A300F208E213F208E213F208E213F208E2137E
:0413B300F208E21347
:1013B700F208E213F208E213F208E213F208E2136A
:1013C700F208E213F29014E1786CE2089313921793
:1013D700E20893139216E20893139215E208931307
:1013E7009214E20893139213E20893139212E208FD
:1013F70093139211E20893139210852266E20893E1
:10140700139217E20893139216E20893139215E2C8
:101417000893139214E20893139213E2089313921A
:1014270012E20893139211E2089313921085226730
:10143700E20893139217E20893139216E2089313A4
:101447009215E20893139214E20893139213E20899
:1014570093139212E20893139211C210852268E542
:1014670066901831856722301602058393602F1422
:10147700F875F003A49016E22582F582E5F035832E
:10148700F583E493F9A3E4939015E1656893C9653F
:10149700679329B401005006885FD233B2A31214B0
:1014A700B7D0F0D0E0D082D083D001D000D0D032F6
:1014B700302F267886E6D5E02076087889E6A2E1FF
:1014C700304401B3923CD239A2E17887E613F6782B
:1014D70088E613F67889E613F6220000000000007C
:1014E70000000000000000000000000000000000F5
:1014F70000000000000000000001000000000000E4
:1015070000000000000000000001000000000000D3
:1015170000010000000100010101000000000000BF
:1015270000000000000000000001000000000000B3
:10153700000100000001000101010000000000009F
:10154700000100000001000101010000000100018D
:10155700010100010101010101010000000000007B
:101567000000000000000000000100000000000073
:10157700000100000001000101010000000000005F
:10158700000100000001000101010000000100014D
:10159700010100010101010101010000000000003B
:1015A700000100000001000101010000000100012D
:1015B7000101000101010101010100000001000119
:1015C7000101000101010101010100010101010106
:1015D70001010101010101010101000101020102F3
:1015E70002030102020302030304010202030203CE
:1015F70003040203030303030405010202030203B6
:10160700030402030304030404050203030403049D
:10161700040503040404040505060102020302038A
:10162700030402030303030404050203030403037F
:101637000405030404050405050602030304030463
:10164700040503040405040505060304040504054D
:10165700050604050506050606070102020302033F
:10166700030402030304030404050203030403043D
:101677000405030404050405050602030304030423
:10168700040503040405040505060304040504050D
:1016970005060405050605060607020303040304F9
:1016A70004050304040504050506030404050405ED
:1016B70005060405050605060607030404050405D3
:1016C70005060405050605060607040505060506BD
:1016D70006070506060706070708FDD00C73700EF8
:1016E7003CF01AAF101E7F9022EC7026D6F02ACB62
:1016F700B02CA3F032BEB03417D03CB6D0461FB0E2
:101707004E77F050F950526AB056DE9058BA306AA8
:10171700CF3072D270745CD076E8F0786BD098E5F1
:10172700709AF8309CBB50A40F70AA7A70B26730D9
:10173700B45DB0B8FCB0C26F50C655D0CA3D90D4A6
:1017470089B0DA94F0DCD790E463B0EA0BF0F431B7
:1017570070F8DD310AB571148FF118D1D126EB512C
:101767002AF6112C8B71463F5148B1F14AACB14C66
:10177700C4F152D9B1546D915A2EF162BD116687E9
:10178700916A9AD16CF29172D5517819F18C71B135
:1017970092D8D19A32D1AA47D1B25A91B452F1C64E
:1017A7007531CC1D71D2A951DCD0B1E85E11EA2B9D
:1017B70011F2EED212F392147D3216973226D8B276
:1017C70032C5F234F7124AEA524C9F5254A5D25806
:1017D7002B725A7552644FD268C1726ADC326C78C8
:0D17E700D2865F128C83729C4EB2A669728E
:1017F400AC1C72B433D2CC18F2EABB330CCE331423
:101804001EB32803F32EE51332F853349873584863
:10181400F36472736845738617B3947313A63C9389
:10182400B221D3B41B53B829B3C641F3D800000086
:1018340000000000000000000000000000000000A4
:10184400000000006A000000000000620D000000BB
:101854000000000000006F004800000000000000CD
:101864000000000000000000006C220000000000E6
:1018740000000000000000000000005B0000000009
:10188400000000000000004100001E475900000055
:10189400260000001D0000100000350000003D007F
:1018A4006B0043000000000000004B000500000036
:1018B40000000000380023000000000000000000C9
:1018C400000000004C0000000000000000000000C8
:1018D40000000000000000000032000004000000CE
:1018E40000000000000000126000370A0000000041
:1018F4000000000000000000080000611346000022
:1019040000000000254D340000572911000000009C
:101914000000640000000000000000000000003A25
:101924004A00002E4F190000001F000000000000B4
:101934006300000000000000270000001B000000FE
:10194400000000000B5F3C006E5D440000006D0071
:101954000000000000000000530000360000283F93
:101964005E00000000000000000300003000700072
:1019740000006900406700000000000055000042BC
:10198400000021000000000000150000000000001D
:101994000000000000005C00170000002000006848
:1019A400020054000E58001C00000000000000005B
:1019B4005A000000000000002F0000002B0000006F
:1019C40000240000006600390000000051000000FF
:1019D4000900520000004500000000000000310032
:1019E40000002A0C000000001A000000000056004D
:1019F40000334E00000000000000000000002C1422
:101A040000003B07003E0000000000000000000052
:101A140000001800001600502D06004900000000C8
:101A24000000000000650F0000000100000000003D
:101A3400000000060000000600060005020600067D
:101A4400000600040406000504020806000000065F
:101A5400000600060006000408060006000600054D
:101A64000806000600021006000600030100000636
:101A740000060002020600060004400600060004F8
:101A84001006000600060006000600060006000513
:101A94001006000600060006000600060001010606
:101AA4000006000600060003020600060000000609
:101AB40000060005010600040202040600060006F2
:101AC4000006000600060006000600048006000268
:101AD40001042006000600060006000600060006B3
:101AE40000060006000600060006000600060006C2
:101AF40000040106000600060006000600031006A6
:101B040000060006000600060006000600060006A1
:101B1400000600060006000308060006000600068C
:0D1B2400000304060006000600060006008F
:10325E00C0E0758400C2CA85CC6F85CD6E75CC007A
:10326E0075CD00D2CA10CF3D20343FE569B4000AB7
:10327E00856E70856F710569802EB4010A856E7238
:10328E00856F7305698021B4020A856E74856F752A
:10329E0005698014B4030E856E76856F77D234750A
:1032AE006900D0E032756900C234D0E032C0D0C0BF
:1032BE00E0C000C001C002C003C004C005C006C00B
:1032CE000730346EAA71AB70AE02AF03EEC40303C7
:1032DE005403FEEFC40303FF54FC4EFEEF5403FFF2
:1032EE00C3E5739AFCE5729BFD50066304FF63050C
:1032FE00FFC3EC9EED9F5038C3E5759AFCE5749BB9
:10330E00FD50066304FF6305FFC3EC9EED9F502046
:10331E00C3E5779AFCE5769BFD50066304FF6305D3
:10332E00FFC3EC9EED9F500885706B85716AD23598
:10333E00C234D007D006D005D004D003D002D001BD
:10334E00D000D0E0D0D02230352F9034A6E56B934C
:10335E00FF9033DA23232582F582E5833400F5834B
:09336E001233B940100F1233B9FB
:10337700400A0F1233B94004C2358004D23622F610
:103387002230352D9034A6E56B93FF9033DA232353
:103397002582F582E5833400F5831233B940100F97
:1033A7001233B9400A0F1233B94004C2358002C242
:1033B7003522E493F9A3E493FAA3E493FBA3E493FC
:1033C700FCA3C3E56A9AE56B995007C3EC956AEBD2
:1033D700956B22EA25DD89DD89D324D324CBD2CB93
:1033E700D2C4DBC4DBBE39BE39B7CAB7CAB18EB1E6
:1033F7008EAB87AB87A59CA59CA000A0009A969A48
:103407009695D895D891E591E58D858D8588AF8876
:10341700AF840C840C7F9A7F9A7B497B49771B7713
:103427001B730F730F6F276F276B576B5767AB674D
:10343700AB642C642C60C660C65D795D795AFE5A10
:10344700FE5970597057E257E25661566154E75476
:10345700E7537453745207520750A050A04F404F80
:10346700404DE64DE64C934C934B414B4149F54952
:10347700F548B548B547764776463E463E45084542
:1034870008432A432A40E440E43F533F533E3E3E2D
:103497003E3C943C943A863A8639183918380532B6
:1034A70032323232323232323232323232323232F5
:1034B70032323232323232323232323232323232E5
:1034C70032323232323232323232323232323232D5
:1034D7003232323232323232313130302F2E2D2DDC
:1034E7002D2C2C2B2A29292827262525242323225E
:1034F7002120201F1E1E1D1C1C1B1A1A1A1A1919FF
:10350700191818181717171716161616151515154B
:10351700141414141313131312121212111111117C
:1035270010101010100F0F0F0F0F0E0E0E0E0E0DA6
:103537000D0D0C0C0C0C0B0B0B0B0B0B0A0A0A0AD0
:103547000A090909090909080808080808070707EF
:103557000707070606060606060605050505050507
:10356700040404040404040303030303030302021F
:10357700020202020201010101010101010101012F
:103587000101010000000000000000000000000031
:0F35970000000000000000000000000000000025
:105731007F011238E17F4C1238B27F541238B27FA8
:10574100521238B27F201238B22055047F308002C5
:105751007F311238B27F201238B29003ADE0784E1B
:10576100123743784E86074307301238B20886074E
:105771004307301238B27507201238B29003AEE0F9
:10578100784E12373B784E86074307301238B208FD
:1057910086074307301238B20886074307301238AC
:1057A100B27507201238B29003ACE0784E1237433D
:1057B100784E86074307301238B208860743073010
:0A57C1001238B27507201238B22228
:106F570044313233343536373839302A23414243C6
:0970DF00126E8B5003126E5C224C
:105DEC00303757E54B540FFF906F5793FE9003F3EA
:105DFC00E475F0011252D4FC740025F0F5827400A5
:105E0C003CF583EEF0EF906F5793FF7895E6062400
:105E1C0096F8A607C2377895E6D394004006125838
:105E2C00D6126E239003F3E0B4030CA3E0B4200766
:105E3C00E49003F3F0A3F0755C02E55C700D7896CA
:0C5E4C00E6642060061258D6126E232275
:106E8B009003F1E0FEA3E0FFA3E0B50607A3E0B596
:066E9B000702C322D3220E
:106C2A009003F1E475F0011252D4FE740025F0F5D8
:106C3A008274003EF583E0FF9003F1E0B4030CA3F5
:0B6C4A00E0B42007E49003F1F0A3F099
:016C5500221C
:106E5C009003F0E014600A14600A240270090267BF
:086E6C0036026F46126D872209
:106736009003E0E0D3940F502E126C2A78A37600D3
:1067460008A6079003E0E02411FF1238E178A4E6DA
:10675600FF9003E0E0FE04F074B12EF582E434030A
:10676600F583EFF00238B275441E9003F0E004F0B2
:016776002200
:106F4600E544700C12390A75440A9003F0E004F027
:016F56002218
:106D8700E544701B7F111238E1126C2A9003B1EFB2
:0F6D9700F01238B29003E07401F0E49003F0F0D2
:016DA60022CA
:106E23007896762008762008762008762008762043
:0E6E3300087620087620087620E47895F6226E
:1058D600E4F584C2997599543099FDC29975993A3F
:1058E6003099FDC2997599203099FDC2997896E64E
:1058F600F5993099FDC2997897E6F5993099FDC2E8
:10590600997898E6F5993099FDC2997899E6F599CE
:105916003099FDC299789AE6F5993099FDC2997841
:105926009BE6F5993099FDC299789CE6F5993099F0
:10593600FDC299789DE6F5993099FDC29975990D44
:0E5946003099FDC29975990A3099FDC29922D7
:10025A0043544353532036332E302020202020206D
:10026A0043544353532036372E3020202020202059
:10027A0043544353532036392E3420202020202043
:10028A0043544353532037312E3920202020202035
:10029A0043544353532037342E3420202020202027
:1002AA0043544353532037372E3020202020202018
:1002BA0043544353532037392E37202020202020FF
:1002CA0043544353532038322E35202020202020F7
:1002DA0043544353532038352E34202020202020E5
:1002EA0043544353532038382E35202020202020D1
:1002FA0043544353532039312E35202020202020C7
:10030A0043544353532039342E38202020202020B0
:10031A0043544353532039372E34202020202020A1
:10032A004354435353203130302E30202020202094
:10033A004354435353203130332E3520202020207C
:10034A004354435353203130372E3220202020206B
:10035A004354435353203131302E3920202020205A
:10036A004354435353203131342E38202020202047
:10037A004354435353203131382E38202020202033
:10038A004354435353203132332E3020202020202F
:10039A004354435353203132372E33202020202018
:1003AA004354435353203133312E38202020202008
:1003BA004354435353203133362E352020202020F6
:1003CA004354435353203134312E332020202020EC
:1003DA004354435353203134362E322020202020D8
:1003EA004354435353203135312E342020202020CA
:1003FA004354435353203135362E372020202020B2
:10040A004354435353203135392E3820202020209D
:10041A004354435353203136322E32202020202099
:10042A004354435353203136352E35202020202083
:10043A004354435353203136372E3920202020206D
:10044A004354435353203137312E33202020202068
:10045A004354435353203137332E38202020202051
:10046A004354435353203137372E33202020202042
:10047A004354435353203137392E3920202020202A
:10048A004354435353203138332E35202020202023
:10049A004354435353203138362E32202020202013
:1004AA004354435353203138392E392020202020F9
:1004BA004354435353203139322E382020202020F0
:1004CA004354435353203139362E362020202020DE
:1004DA004354435353203139392E352020202020CC
:1004EA004354435353203230332E352020202020CA
:1004FA004354435353203230362E352020202020B7
:10050A004354435353203231302E372020202020A9
:10051A004354435353203231382E31202020202097
:10052A004354435353203232352E37202020202083
:10053A004354435353203232392E31202020202075
:10054A004354435353203233332E36202020202065
:10055A004354435353203234312E38202020202054
:10056A004354435353203235302E33202020202049
:10057A004354435353203235342E31202020202037
:10058A002020202020202020202020202020202061
:10059A004443532030303620494E562030323120E1
:1005AA004443532030303720494E562032313420CC
:1005BA004443532030313520494E562031343120BE
:1005CA004443532030313720494E562030353020AD
:1005DA004443532030323120494E562030303620A1
:1005EA004443532030323320494E5620303437208A
:1005FA004443532030323520494E56203234342079
:10060A004443532030323620494E56203436342063
:10061A004443532030333120494E56203632372056
:10062A004443532030333220494E5620303531204E
:10063A004443532030333620494E56203137322036
:10064A004443532030343320494E56203434352025
:10065A004443532030343720494E56203032332019
:10066A004443532030353020494E5620303137200C
:10067A004443532030353120494E562030333220FE
:10068A004443532030353320494E562034353220E6
:10069A004443532030353420494E562034313320D8
:1006AA004443532030363520494E562032373120C4
:1006BA004443532030373120494E562033303620B8
:1006CA004443532030373220494E562032343520A5
:1006DA004443532030373320494E56203530362094
:1006EA004443532030373420494E56203137342082
:1006FA004443532031313420494E56203731322079
:10070A004443532031313520494E56203135322069
:10071A004443532031313620494E56203735342050
:10072A004443532031323220494E5620323235204A
:10073A004443532031323520494E56203336352032
:10074A004443532031333120494E56203336342026
:10075A004443532031333220494E56203534362013
:10076A004443532031333420494E56203232332009
:10077A004443532031343120494E562030313520FC
:10078A004443532031343320494E562034313220E9
:10079A004443532031343520494E562032373420D1
:1007AA004443532031353220494E562031313520C9
:1007BA004443532031353520494E562037333120B2
:1007CA004443532031353620494E5620323635209F
:1007DA004443532031363220494E56203530332097
:1007EA004443532031363520494E56203235312084
:1007FA004443532031373220494E56203033362075
:10080A004443532031373420494E56203037342060
:10081A004443532032303520494E56203236332055
:10082A004443532032313220494E56203335362044
:10083A004443532032313420494E56203030372039
:10084A004443532032323320494E56203133342028
:10085A004443532032323520494E56203132322019
:10086A004443532032323620494E56203431312007
:10087A004443532032343320494E562033353120F5
:10088A004443532032343420494E562030323520E6
:10089A004443532032343520494E562030373220D3
:1008AA004443532032343620494E562035323320C1
:1008BA004443532032353120494E562031363520B3
:1008CA004443532032353220494E562034363220A2
:1008DA004443532032353520494E5620343436208D
:1008EA004443532032363120494E56203733322082
:1008FA004443532032363320494E56203230352075
:10090A004443532032363520494E5620313536205D
:10091A004443532032363620494E5620343534204B
:10092A004443532032373120494E56203036352041
:10093A004443532032373420494E5620313435202F
:10094A004443532033303620494E56203037312025
:10095A004443532033313120494E56203636342011
:10096A004443532033313520494E56203432332004
:10097A004443532033323520494E562035323620EF
:10098A004443532033333120494E562034363520E0
:10099A004443532033333220494E562034353520D0
:1009AA004443532033343320494E562035333220C2
:1009BA004443532033343620494E562036313220B0
:1009CA004443532033353120494E562032343320A4
:1009DA004443532033353620494E56203231322093
:1009EA004443532033363420494E56203133312084
:1009FA004443532033363520494E56203132352070
:100A0A004443532033373120494E5620373334205C
:100A1A004443532034313120494E56203232362055
:100A2A004443532034313220494E56203134332046
:100A3A004443532034313320494E56203035342034
:100A4A004443532034323320494E56203331352023
:100A5A004443532034333120494E56203732332011
:100A6A004443532034333220494E56203531362000
:100A7A004443532034343520494E562030343320F1
:100A8A004443532034343620494E562032353520DB
:100A9A004443532034353220494E562030353320D2
:100AAA004443532034353420494E562032363620BA
:100ABA004443532034353520494E562033333220AF
:100ACA004443532034363220494E562032353220A0
:100ADA004443532034363420494E5620303236208F
:100AEA004443532034363520494E5620333331207F
:100AFA004443532034363620494E56203636322067
:100B0A004443532035303320494E56203136322063
:100B1A004443532035303620494E5620303733204F
:100B2A004443532035313620494E5620343332203F
:100B3A004443532035323320494E5620323436202E
:100B4A004443532035323620494E5620333235201D
:100B5A004443532035333220494E56203334332010
:100B6A004443532035343620494E562031333220FF
:100B7A004443532035363520494E562037303320EA
:100B8A004443532036303620494E562036333120DE
:100B9A004443532036313220494E562033343620CE
:100BAA004443532036323420494E562036333220BD
:100BBA004443532036323720494E562030333120B1
:100BCA004443532036333120494E5620363036209E
:100BDA004443532036333220494E5620363234208D
:100BEA004443532036353420494E56203734332077
:100BFA004443532036363220494E56203436362066
:100C0A004443532036363420494E5620333131205E
:100C1A004443532037303320494E56203536352049
:100C2A004443532037313220494E56203131342043
:100C3A004443532037323320494E5620343331202F
:100C4A004443532037333120494E5620313535201D
:100C5A004443532037333220494E5620323631200E
:100C6A004443532037333420494E562033373120FA
:100C7A004443532037343320494E562036353420E6
:100C8A004443532037353420494E562031313620DB
:100C9A003030362030323130303720323134303152
:100CAA00352031343130313720303530303231204F
:100CBA003030363032332030343730323520323427
:100CCA00343032362034363430333120363237300D
:100CDA003332203035313033362031373230343305
:100CEA002034343530343720303233303530203008
:100CFA0031373035312030333230353320343532E4
:100D0A0030353420343133303635203237313037CC
:100D1A0031203330363037322032343530373320D1
:100D2A0035303630373420313734313134203731A9
:100D3A00323131352031353231313620373534319F
:100D4A003232203232353132352033363531333191
:100D5A00203336343133322035343631333420328D
:100D6A003233313431203031353134332034313279
:100D7A00313435203237343135322031313531355D
:100D8A003520373331313536203236353136322057
:100D9A003530333136352032353131373220303340
:100DAA003631373420303734323035203236333228
:100DBA003132203335363231342030303732323323
:100DCA002031333432323520313232323236203425
:100DDA003131323433203335313234342030323504
:100DEA0032343520303732323436203532333235E8
:100DFA0031203136353235322034363232353520EB
:100E0A0034343632363120373332323633203230C8
:100E1A0035323635203135363236362034353432AD
:100E2A0037312030363532373420313435333036A5
:100E3A0020303731333131203636343331352034AE
:100E4A003233333235203532363333312034363586
:100E5A003333322034353533343320353332333477
:100E6A003620363132333531203234333335362079
:100E7A003231323336342031333133363520313260
:100E8A003533373120373334343131203232363446
:100E9A003132203134333431332030353434323343
:100EAA00203331353433312037323334333220353D
:100EBA003136343435203034333434362032353513
:100ECA003435322030353334353420323636343501
:100EDA003520333332343632203235323436342008
:100EEA0030323634363520333331343636203636DE
:100EFA0032353033203136323530362030373335DB
:100F0A0031362034333235323320323436353236C4
:100F1A0020333235353332203334333534362031C9
:100F2A0033323536352037303336303620363331A2
:100F3A003631322033343636323420363332363292
:100F4A00372030333136333120363036363332209B
:100F5A003632343635342037343336363220343666
:100F6A00363636342033313137303320353635375B
:100F7A00313220313134373233203433313733315F
:100F8A002031353537333220323631373334203356
:100F9A00373137343320363534373534203131362A
:100FAA00203633302036373020363934203731393D
:100FBA002037343420373730203739372038323524
:100FCA00203835342038383520393135203934380D
:100FDA0020393734313030303130333531303732EF
:100FEA0031313039313134383131383831323330C6
:100FFA0031323733313331383133363531343133B5
:10100A003134363231353134313536373135393894
:10101A003136323231363535313637393137313387
:10102A003137333831373733313739393138333566
:10103A003138363231383939313932383139363650
:10104A00313939353230333532303635323130375D
:10105A00323138313232353732323931323333364E
:0C106A0032343138323530333235343115
:105F91007890E6B41200505D905FA0F82828730253
:105FA1005FD6025FE8025FD9025FE8025FDC025F51
:105FB100E8025FDE025FE8025FE0025FE8025FE2A3
:105FC100025FE8025FE5025FE8025FEA025FE80262
:105FD1005FF0025FF3026DA7026FCD80078005803D
:105FE10003027085026C56800302708F02703F02BB
:065FF1007099126FA3225B
:106DA7007893E675F010A4245AF9740235F0FA7B4B
:106DB700FF126B43E4F584C29975994378900622D4
:0C703F00E4F584309905789006C299228F
:0D6FCD00E4F58475993A7891F678900622E3
:106C5600E4F5847891E606FF7893E625E025E024BE
:106C6600AAF582E4340FF583E5822FF582E43583B5
:0A6C7600F583E493F5997890062267
:0A708500E4F58475992E7890062238
:0A708F00E4F58475990D789006224F
:0A709900E4F58475990A7890062248
:0E6FA300E4F5843099077890F6C299C25A221C
:105C2B00788EE6B41600506C905C3AF82828730214
:105C3B005C7C025C91025C7F025C91025C82025C88
:105C4B0091025C84025C91025C86025C91025C882E
:105C5B00025C91025C8A025C91025C8C025C910298
:105C6B005C8E025C91025C93025C91025C99025C1B
:105C7B009C026DE6026FDA800A8008800680048041
:105C8B00028000026C8080030270A302704B0270D2
:055C9B00AD126FB12203
:106DE600E55F75F010A4249AF9740535F0FA7BFF77
:0F6DF600126B43E4F584C299759944788E062296
:0C704B00E4F584309905788E06C2992285
:0D6FDA00E4F58475993A788FF6788E0622DA
:106C8000E4F584788FE606FF75F007E55FA4249AA3
:106C9000F582E5F0340CF583E5822FF582E4358347
:0A6CA000F583E493F599788E06223F
:0A70A300E4F58475990D788E06223D
:0A70AD00E4F58475990A788E062236
:0E6FB100E4F584309907788EF6C299C25B220F
:1055F4007892E6B41E004003025693905606F828AB
:105604002873025660025685025663025685025676
:105614006602568502566902568502566B02568505
:1056240002566E0256850256710256850256730260
:1056340056850256760256850256790256850256DA
:105644007C02568502567F02568502568202568592
:1056540002568702568502568D025690026F9402B6
:1056640070B7026F348011026EF5026FE780090291
:105674006F0A026FF40270010270C1026F1F0270A0
:105684000E80030270CB0270570270D5126FBF22D6
:0F6F9400125731E4F584C29975994C7892062210
:0C705700E4F584309905789206C2992275
:0A70B700E4F58475993A78920622F8
:106F3400E4F584305505759931800375993078925C
:026F4400062223
:0A70C100E4F5847599207892062208
:106EF5009003ADE0FF123680E4F5849003C2E0F51F
:056F05009978920622BC
:0D6FE700E4F5849003C3E0F599789206224A
:106F0A009003AEE0FF123680E4F5849003C1E0F509
:056F1A009978920622A7
:0D6FF400E4F5849003C2E0F599789206223E
:0D700100E4F5849003C3E0F599789206222F
:106F1F009003ACE0FF123680E4F5849003C2E0F5F5
:056F2F00997892062292
:0D700E00E4F5849003C3E0F5997892062222
:0A70CB00E4F58475990D7892062211
:0A70D500E4F58475990A789206220A
:0E6FBF00E4F5843099077892F6C299C25C22FC
:0300000002706328
:0C706300787FE4F6D8FD7581A4024F751B
:10525200BB010CE58229F582E5833AF583E0225011
:1052620006E92582F8E622BBFE06E92582F8E2225B
:0D527200E58229F582E5833AF583E4932275
:10527F00BC000BBE0029EF8DF084FFADF022E4CC13
:10528F00F875F008EF2FFFEE33FEEC33FCEE9DECDC
:10529F00984005FCEE9DFE0FD5F0E9E4CEFD22ED22
:1052AF00F8F5F0EE8420D21CFEADF075F008EF2F6C
:1052BF00FFED33FD4007985006D5F0F222C398FD5D
:0552CF000FD5F0EA22FA
:1052D400A3F8E0C5F025F0F0E5821582700215838D
:0652E400E0C838F0E822EA
:0C52EA00A42582F582E5F03583F58322CF
:1052F600D083D082F8E4937012740193700DA3A347
:1053060093F8740193F5828883E47374029368605A
:06531600EFA3A3A380DF5A
:00000001FF
